LX51 LINKER/LOCATER V4.66.97.0                                                          03/28/2025  17:08:22  PAGE 1


LX51 LINKER/LOCATER V4.66.97.0, INVOKED BY:
C:\KEIL_V5\C51\BIN\LX51.EXE .\Out_Files\STARTUP.obj, .\Out_Files\system_um800xx.obj, .\Out_Files\common.obj, .\Out_Files
>> \eflash.obj, .\Out_Files\uart0.obj, .\Out_Files\app.obj, .\Out_Files\main.obj TO .\Out_Files\EFLASH_Example PRINT (.\
>> Out_Files\EFLASH_Example.map) REMOVEUNUSED CLASSES (XDATA (X:0X0-X:0X7FF), HDATA (X:0X0-X:0X7FF), ECODE (C:0X0-C:0XFF
>> FF), HCONST (C:0X0-C:0XFFFF))


CPU MODE:     8051 MODE
MEMORY MODEL: LARGE


INPUT MODULES INCLUDED:
  .\Out_Files\STARTUP.obj (?C_STARTUP)
         COMMENT TYPE 1: A51 / ASM51 Assembler
  .\Out_Files\system_um800xx.obj (SYSTEM_UM800XX)
         COMMENT TYPE 0: C51 V9.60.0.0
  .\Out_Files\common.obj (COMMON)
         COMMENT TYPE 0: C51 V9.60.0.0
  .\Out_Files\eflash.obj (EFLASH)
         COMMENT TYPE 0: C51 V9.60.0.0
  .\Out_Files\uart0.obj (UART0)
         COMMENT TYPE 0: C51 V9.60.0.0
  .\Out_Files\app.obj (APP)
         COMMENT TYPE 0: C51 V9.60.0.0
  .\Out_Files\main.obj (MAIN)
         COMMENT TYPE 0: C51 V9.60.0.0
  C:\KEIL_V5\C51\LIB\C51L.LIB (?C_INIT)
         COMMENT TYPE 1: A51 / ASM51 Assembler
  C:\KEIL_V5\C51\LIB\C51L.LIB (?C?CLDPTR)
         COMMENT TYPE 1: A51 / ASM51 Assembler
  C:\KEIL_V5\C51\LIB\C51L.LIB (?C?CLDOPTR)
         COMMENT TYPE 1: A51 / ASM51 Assembler
  C:\KEIL_V5\C51\LIB\C51L.LIB (?C?CSTPTR)
         COMMENT TYPE 1: A51 / ASM51 Assembler
  C:\KEIL_V5\C51\LIB\C51L.LIB (?C?CSTOPTR)
         COMMENT TYPE 1: A51 / ASM51 Assembler
  C:\KEIL_V5\C51\LIB\C51L.LIB (?C?IILDX)
         COMMENT TYPE 1: A51 / ASM51 Assembler
  C:\KEIL_V5\C51\LIB\C51L.LIB (?C?ILDIX)
         COMMENT TYPE 1: A51 / ASM51 Assembler
  C:\KEIL_V5\C51\LIB\C51L.LIB (?C?LADD)
         COMMENT TYPE 1: A51 / ASM51 Assembler
  C:\KEIL_V5\C51\LIB\C51L.LIB (?C?LMUL)
         COMMENT TYPE 1: A51 / ASM51 Assembler
  C:\KEIL_V5\C51\LIB\C51L.LIB (?C?ULDIV)
         COMMENT TYPE 1: A51 / ASM51 Assembler
  C:\KEIL_V5\C51\LIB\C51L.LIB (?C?LOR)
         COMMENT TYPE 1: A51 / ASM51 Assembler
  C:\KEIL_V5\C51\LIB\C51L.LIB (?C?ULCMP)
         COMMENT TYPE 1: A51 / ASM51 Assembler
  C:\KEIL_V5\C51\LIB\C51L.LIB (?C?ULSHR)
         COMMENT TYPE 1: A51 / ASM51 Assembler
  C:\KEIL_V5\C51\LIB\C51L.LIB (?C?LSHL)
         COMMENT TYPE 1: A51 / ASM51 Assembler
  C:\KEIL_V5\C51\LIB\C51L.LIB (?C?LLDOPTR)
         COMMENT TYPE 1: A51 / ASM51 Assembler
  C:\KEIL_V5\C51\LIB\C51L.LIB (?C?LLDXDATA)
         COMMENT TYPE 1: A51 / ASM51 Assembler
  C:\KEIL_V5\C51\LIB\C51L.LIB (?C?LLDXDATA0)
         COMMENT TYPE 1: A51 / ASM51 Assembler
  C:\KEIL_V5\C51\LIB\C51L.LIB (?C?LLDIXDATA)
         COMMENT TYPE 1: A51 / ASM51 Assembler
  C:\KEIL_V5\C51\LIB\C51L.LIB (?C?LSTXDATA)
         COMMENT TYPE 1: A51 / ASM51 Assembler
  C:\KEIL_V5\C51\LIB\C51L.LIB (?C?LSTKXDATA)
         COMMENT TYPE 1: A51 / ASM51 Assembler
LX51 LINKER/LOCATER V4.66.97.0                                                        03/28/2025  17:08:22  PAGE 2


  C:\KEIL_V5\C51\LIB\C51L.LIB (?C?PLDXDATA)
         COMMENT TYPE 1: A51 / ASM51 Assembler
  C:\KEIL_V5\C51\LIB\C51L.LIB (?C?PLDIXDATA)
         COMMENT TYPE 1: A51 / ASM51 Assembler
  C:\KEIL_V5\C51\LIB\C51L.LIB (?C?PSTXDATA)
         COMMENT TYPE 1: A51 / ASM51 Assembler
  C:\KEIL_V5\C51\LIB\C51L.LIB (?C?LCASE)
         COMMENT TYPE 1: A51 / ASM51 Assembler
  C:\KEIL_V5\C51\LIB\C51L.LIB (?C?ICALL)
         COMMENT TYPE 1: A51 / ASM51 Assembler
  C:\KEIL_V5\C51\LIB\C51L.LIB (PRINTF)
         COMMENT TYPE 1: A51 / ASM51 Assembler
  C:\KEIL_V5\C51\LIB\C51L.LIB (?C?LLDIDATA)
         COMMENT TYPE 1: A51 / ASM51 Assembler
  C:\KEIL_V5\C51\LIB\C51L.LIB (?C?LLDPDATA)
         COMMENT TYPE 1: A51 / ASM51 Assembler
  C:\KEIL_V5\C51\LIB\C51L.LIB (?C?LLDCODE)
         COMMENT TYPE 1: A51 / ASM51 Assembler
  C:\KEIL_V5\C51\LIB\C51L.LIB (?C?CCASE)
         COMMENT TYPE 1: A51 / ASM51 Assembler


ACTIVE MEMORY CLASSES OF MODULE:  .\Out_Files\EFLASH_Example (?C_STARTUP)

BASE        START       END         USED      MEMORY CLASS
==========================================================
X:000000H   X:000000H   X:0007FFH   0000C8H   XDATA
X:000000H   X:000000H   X:0007FFH             HDATA
C:000000H   C:000000H   C:00FFFFH             ECODE
C:000000H   C:000000H   C:00FFFFH             HCONST
C:000000H   C:000000H   C:00FFFFH   001149H   CODE
I:000000H   I:000000H   I:0000FFH   000001H   IDATA
C:000000H   C:000000H   C:00FFFFH   000233H   CONST
I:000020H.0 I:000020H.0 I:00002FH.7 000001H.1 BIT
I:000000H   I:000000H   I:00007FH   00000DH   DATA


MEMORY MAP OF MODULE:  .\Out_Files\EFLASH_Example (?C_STARTUP)


START     STOP      LENGTH    ALIGN  RELOC    MEMORY CLASS   SEGMENT NAME
=========================================================================

* * * * * * * * * * *   D A T A   M E M O R Y   * * * * * * * * * * * * *
000000H   000007H   000008H   ---    AT..     DATA           "REG BANK 0"
000008H   00000CH   000005H   BYTE   UNIT     DATA           _DATA_GROUP_
00000DH.0 00001FH.7 000013H.0 ---    ---      **GAP**
000020H.0 000021H.0 000001H.1 BIT    UNIT     BIT            _BIT_GROUP_
000021H.1 000021H   000000H.7 ---    ---      **GAP**
000022H   000022H   000001H   BYTE   UNIT     IDATA          ?STACK

* * * * * * * * * * *   C O D E   M E M O R Y   * * * * * * * * * * * * *
000000H   000002H   000003H   ---    OFFS..   CODE           ?CO??C_STARTUP?0
000003H   00001BH   000019H   BYTE   UNIT     CODE           ?PR?UART_INIT?APP
00001CH   000020H   000005H   BYTE   UNIT     CODE           ?PR?_PUTCHAR?UART0
000021H   000022H   000002H   ---    ---      **GAP**
000023H   000025H   000003H   BYTE   OFFS..   CODE           ?UART0?00023
000026H   0003AAH   000385H   BYTE   UNIT     CODE           ?C?LIB_CODE
0003ABH   00070FH   000365H   BYTE   UNIT     CODE           ?PR?PRINTF?PRINTF
000710H   0008C0H   0001B1H   BYTE   UNIT     CODE           ?PR?_EFLASH_PAGE_CHECK_BYTES?APP
0008C1H   000A03H   000143H   BYTE   UNIT     CODE           ?PR?_CLOCK_INIT?SYSTEM_UM800XX
000A04H   000AC9H   0000C6H   BYTE   UNIT     CODE           ?PR?_READ_UID?EFLASH
000ACAH   000B77H   0000AEH   BYTE   UNIT     CODE           ?PR?_EFLASH_PAGE_CHECK_BYTE?APP
000B78H   000C16H   00009FH   BYTE   UNIT     CODE           ?PR?EFLASH_SN_TEST?APP
000C17H   000CB0H   00009AH   BYTE   UNIT     CODE           ?C_C51STARTUP
LX51 LINKER/LOCATER V4.66.97.0                                                        03/28/2025  17:08:22  PAGE 3


000CB1H   000D28H   000078H   BYTE   UNIT     CODE           ?PR?_EFLASH_READ_BYTES?EFLASH
000D29H   000D9FH   000077H   BYTE   UNIT     CODE           ?PR?_UART0_SET_BAUD_RATE?UART0
000DA0H   000E0CH   00006DH   BYTE   UNIT     CODE           ?PR?EFLASH_TEST?APP
000E0DH   000E78H   00006CH   BYTE   UNIT     CODE           ?PR?_PRINTF_BUFF_BYTE?COMMON
000E79H   000EDDH   000065H   BYTE   UNIT     CODE           ?PR?_EFLASH_WRITE_BYTES?EFLASH
000EDEH   000F33H   000056H   BYTE   UNIT     CODE           ?PR?_READ_VCAP?EFLASH
000F34H   000F84H   000051H   BYTE   UNIT     CODE           ?C_INITSEG
000F85H   000FCEH   00004AH   BYTE   UNIT     CODE           ?PR?UART0_IRQHANDLER?UART0
000FCFH   001015H   000047H   BYTE   UNIT     CODE           ?PR?_DELAY1MS?COMMON
001016H   00104CH   000037H   BYTE   UNIT     CODE           ?PR?_UART0_INIT?UART0
00104DH   001080H   000034H   BYTE   UNIT     CODE           ?PR?_EFLASH_INIT?EFLASH
001081H   0010B1H   000031H   BYTE   UNIT     CODE           ?PR?_READ_SEQUENCE?EFLASH
0010B2H   0010DFH   00002EH   BYTE   UNIT     CODE           ?PR?_EFLASH_ERASE_PAGE?EFLASH
0010E0H   001101H   000022H   BYTE   UNIT     CODE           ?PR?UART0_REC_PRO?APP
001102H   001117H   000016H   BYTE   UNIT     CODE           ?PR?_UART0_SEND_BYTE?UART0
001118H   001129H   000012H   BYTE   UNIT     CODE           ?PR?_UART0_IRQ_INIT?UART0
00112AH   001134H   00000BH   BYTE   UNIT     CODE           ?PR?SYSTEM_INIT?SYSTEM_UM800XX
001135H   00113FH   00000BH   BYTE   UNIT     CODE           ?PR?MAIN?MAIN
001140H   001147H   000008H   BYTE   UNIT     CODE           ?PR?_EFLASH_READ_BYTE?EFLASH
001148H   00114AH   000003H   BYTE   UNIT     CODE           ?PR?UART0_RECV_BYTE?UART0
00114BH   00136DH   000223H   BYTE   UNIT     CONST          ?CO?APP
00136EH   00137DH   000010H   BYTE   UNIT     CONST          ?CO?COMMON

* * * * * * * * * * *  X D A T A   M E M O R Y  * * * * * * * * * * * * *
000000H   00006CH   00006DH   BYTE   UNIT     XDATA          ?XD?APP
00006DH   0000BBH   00004FH   BYTE   UNIT     XDATA          _XDATA_GROUP_
0000BCH   0000C3H   000008H   BYTE   UNIT     XDATA          ?XD?SYSTEM_UM800XX
0000C4H   0000C7H   000004H   BYTE   UNIT     XDATA          ?XD?UART0

* * * * * * * * *   R E M O V E D     S E G M E N T S   * * * * * * * *
   *DEL*:           000015H   BYTE   UNIT     CODE           ?PR?_DELAY?COMMON
   *DEL*:           000004H   BYTE   UNIT     XDATA          ?XD?_DELAY?COMMON
   *DEL*:           000077H   BYTE   UNIT     CODE           ?PR?_PRINTF_BUFF_WORD?COMMON
   *DEL*:           00000BH   BYTE   UNIT     XDATA          ?XD?_PRINTF_BUFF_WORD?COMMON
   *DEL*:           000032H   BYTE   UNIT     CODE           ?PR?_EFLASH_WRITE_BYTE?EFLASH
   *DEL*:           000000H.1 BIT    UNIT     BIT            ?BI?_EFLASH_WRITE_BYTE?EFLASH
   *DEL*:           00002EH   BYTE   UNIT     CODE           ?PR?_UART0_SEND_BYTES?UART0
   *DEL*:           000007H   BYTE   UNIT     XDATA          ?XD?_UART0_SEND_BYTES?UART0
   *DEL*:           0000F3H   BYTE   UNIT     CODE           ?PR?_EFLASH_PAGE_CHECK_8BITS?APP
   *DEL*:           000006H   BYTE   UNIT     XDATA          ?XD?_EFLASH_PAGE_CHECK_8BITS?APP



OVERLAY MAP OF MODULE:   .\Out_Files\EFLASH_Example (?C_STARTUP)


FUNCTION/MODULE                    BIT_GROUP   DATA_GROUP   XDATA_GROUP
--> CALLED FUNCTION/MODULE        START  STOP  START  STOP  START  STOP
=======================================================================
?C_C51STARTUP                     ----- -----  ----- -----  ----- -----
  +--> MAIN/MAIN
  +--> ?C_INITSEG

MAIN/MAIN                         ----- -----  ----- -----  ----- -----
  +--> SYSTEM_INIT/SYSTEM_UM800XX
  +--> UART_INIT/APP
  +--> EFLASH_TEST/APP

SYSTEM_INIT/SYSTEM_UM800XX        ----- -----  ----- -----  ----- -----
  +--> _CLOCK_INIT/SYSTEM_UM800XX

_CLOCK_INIT/SYSTEM_UM800XX        ----- -----  ----- -----  006DH 0074H

UART_INIT/APP                     ----- -----  ----- -----  ----- -----
  +--> _UART0_INIT/UART0
LX51 LINKER/LOCATER V4.66.97.0                                                        03/28/2025  17:08:22  PAGE 4


  +--> UART0_REC_PRO/APP
  +--> _UART0_IRQ_INIT/UART0

_UART0_INIT/UART0                 ----- -----  ----- -----  006DH 0070H
  +--> _UART0_SET_BAUD_RATE/UART0

_UART0_SET_BAUD_RATE/UART0        ----- -----  ----- -----  0071H 007CH

UART0_REC_PRO/APP                 ----- -----  ----- -----  ----- -----
  +--> UART0_RECV_BYTE/UART0

UART0_RECV_BYTE/UART0             ----- -----  ----- -----  ----- -----

_UART0_IRQ_INIT/UART0             ----- -----  ----- -----  ----- -----

EFLASH_TEST/APP                   ----- -----  ----- -----  ----- -----
  +--> PRINTF/PRINTF
  +--> _EFLASH_INIT/EFLASH
  +--> _EFLASH_PAGE_CHECK_BYTE/APP
  +--> _DELAY1MS/COMMON
  +--> _EFLASH_PAGE_CHECK_BYTES/APP
  +--> EFLASH_SN_TEST/APP

PRINTF/PRINTF                     20H.0 21H.0  0008H 000CH  0094H 00BBH
  +--> _PUTCHAR/UART0

_PUTCHAR/UART0                    ----- -----  ----- -----  ----- -----
  +--> _UART0_SEND_BYTE/UART0

_UART0_SEND_BYTE/UART0            ----- -----  ----- -----  ----- -----

_EFLASH_INIT/EFLASH               ----- -----  ----- -----  006DH 0070H

_EFLASH_PAGE_CHECK_BYTE/APP       ----- -----  ----- -----  006DH 0072H
  +--> _EFLASH_ERASE_PAGE/EFLASH
  +--> _EFLASH_READ_BYTE/EFLASH
  +--> PRINTF/PRINTF

_EFLASH_ERASE_PAGE/EFLASH         20H.0 20H.0  ----- -----  ----- -----

_EFLASH_READ_BYTE/EFLASH          ----- -----  ----- -----  ----- -----

_DELAY1MS/COMMON                  ----- -----  ----- -----  006DH 0074H

_EFLASH_PAGE_CHECK_BYTES/APP      ----- -----  ----- -----  006DH 0077H
  +--> _EFLASH_ERASE_PAGE/EFLASH
  +--> _EFLASH_READ_BYTE/EFLASH
  +--> PRINTF/PRINTF
  +--> _EFLASH_WRITE_BYTES/EFLASH
  +--> _EFLASH_READ_BYTES/EFLASH

_EFLASH_WRITE_BYTES/EFLASH        20H.0 20H.0  ----- -----  0078H 0080H

_EFLASH_READ_BYTES/EFLASH         ----- -----  ----- -----  0078H 0084H

EFLASH_SN_TEST/APP                ----- -----  ----- -----  006DH 0088H
  +--> PRINTF/PRINTF
  +--> _READ_SEQUENCE/EFLASH
  +--> _PRINTF_BUFF_BYTE/COMMON
  +--> _READ_UID/EFLASH
  +--> _READ_VCAP/EFLASH

_READ_SEQUENCE/EFLASH             ----- -----  ----- -----  0089H 008BH

_PRINTF_BUFF_BYTE/COMMON          ----- -----  ----- -----  0089H 0093H
LX51 LINKER/LOCATER V4.66.97.0                                                        03/28/2025  17:08:22  PAGE 5


  +--> PRINTF/PRINTF

_READ_UID/EFLASH                  ----- -----  ----- -----  0089H 008CH

_READ_VCAP/EFLASH                 ----- -----  ----- -----  0089H 008CH

?C_INITSEG                        ----- -----  ----- -----  ----- -----

*** NEW ROOT ********************

UART0_IRQHANDLER/UART0            ----- -----  ----- -----  ----- -----



PUBLIC SYMBOLS OF MODULE:  .\Out_Files\EFLASH_Example (?C_STARTUP)


      VALUE       CLASS    TYPE      PUBLIC SYMBOL NAME
      =================================================
      0200006DH   XDATA    BYTE      ?_eflash_page_check_bytes?BYTE
      02000078H   XDATA    BYTE      ?_eflash_read_bytes?BYTE
      02000078H   XDATA    BYTE      ?_eflash_write_bytes?BYTE
      02000094H   XDATA    ---       ?_PRINTF517?BYTE
      02000094H   XDATA    ---       ?_PRINTF?BYTE
      02000094H   XDATA    ---       ?_SPRINTF517?BYTE
      02000094H   XDATA    ---       ?_SPRINTF?BYTE
      01000385H   CODE     ---       ?C?CCASE
      0100003FH   CODE     ---       ?C?CLDOPTR
      01000026H   CODE     ---       ?C?CLDPTR
      00000000H   NUMBER   ---       ?C?CODESEG
      0100007EH   CODE     ---       ?C?CSTOPTR
      0100006CH   CODE     ---       ?C?CSTPTR
      01000357H   CODE     ---       ?C?ICALL
      0100035BH   CODE     ---       ?C?ICALL2
      010000A0H   CODE     ---       ?C?IILDX
      010000B6H   CODE     ---       ?C?ILDIX
      010000CCH   CODE     ---       ?C?LADD
      0100031DH   CODE     ---       ?C?LCASE
      01000375H   CODE     ---       ?C?LLDCODE
      0100035DH   CODE     ---       ?C?LLDIDATA
      0100028BH   CODE     ---       ?C?LLDIXDATA
      01000282H   CODE     ---       ?C?LLDIXDATA1
      01000284H   CODE     ---       ?C?LLDIXDATA8
      0100023AH   CODE     ---       ?C?LLDOPTR
      01000369H   CODE     ---       ?C?LLDPDATA
      0100026AH   CODE     ---       ?C?LLDXDATA
      01000276H   CODE     ---       ?C?LLDXDATA0
      010000D9H   CODE     ---       ?C?LMUL
      010001F6H   CODE     ---       ?C?LOR
      01000227H   CODE     ---       ?C?LSHL
      010002C3H   CODE     ---       ?C?LSTKXDATA
      010002B7H   CODE     ---       ?C?LSTXDATA
      010002FDH   CODE     ---       ?C?PLDIXDATA
      010002F4H   CODE     ---       ?C?PLDXDATA
      01000314H   CODE     ---       ?C?PSTXDATA
      01000203H   CODE     ---       ?C?ULCMP
      01000164H   CODE     ---       ?C?ULDIV
      01000214H   CODE     ---       ?C?ULSHR
      00000000H   NUMBER   ---       ?C?XDATASEG
      01000C6CH   CODE     ---       ?C_START
      01000000H   CODE     ---       ?C_STARTUP
      010008C1H   CODE     ---       _clock_init
*DEL*:00000000H   CODE     ---       _delay
      01000FCFH   CODE     ---       _delay1ms
      010010B2H   CODE     ---       _eflash_erase_page
LX51 LINKER/LOCATER V4.66.97.0                                                        03/28/2025  17:08:22  PAGE 6


      0100104DH   CODE     ---       _eflash_init
*DEL*:00000000H   CODE     ---       _eflash_page_check_8bits
      01000ACAH   CODE     ---       _eflash_page_check_byte
      01000710H   CODE     ---       _eflash_page_check_bytes
      01001140H   CODE     ---       _eflash_read_byte
      01000CB1H   CODE     ---       _eflash_read_bytes
*DEL*:00000000H   CODE     ---       _eflash_write_byte
      01000E79H   CODE     ---       _eflash_write_bytes
      01000416H   CODE     ---       _PRINTF
      01000416H   CODE     ---       _PRINTF517
      01000E0DH   CODE     ---       _printf_buff_byte
*DEL*:00000000H   CODE     ---       _printf_buff_word
      0100001CH   CODE     ---       _putchar
      01001081H   CODE     ---       _read_sequence
      01000A04H   CODE     ---       _read_UID
      01000EDEH   CODE     ---       _read_Vcap
      01000410H   CODE     ---       _SPRINTF
      01000410H   CODE     ---       _SPRINTF517
      01001016H   CODE     ---       _uart0_init
      01001118H   CODE     ---       _uart0_irq_init
      01001102H   CODE     ---       _uart0_send_byte
*DEL*:00000000H   CODE     ---       _uart0_send_bytes
*SFR* 000000D0H.6 DATA     BIT       AC
*SFR* 000000E0H   DATA     BYTE      ACC
*SFR* 000000E0H.0 DATA     BIT       ACC0
*SFR* 000000E0H.1 DATA     BIT       ACC1
*SFR* 000000E0H.2 DATA     BIT       ACC2
*SFR* 000000E0H.3 DATA     BIT       ACC3
*SFR* 000000E0H.4 DATA     BIT       ACC4
*SFR* 000000E0H.5 DATA     BIT       ACC5
*SFR* 000000E0H.6 DATA     BIT       ACC6
*SFR* 000000E0H.7 DATA     BIT       ACC7
*SFR* 000000FEH   DATA     BYTE      ADCCDR0
*SFR* 000000FFH   DATA     BYTE      ADCCDR1
*SFR* 000000F6H   DATA     BYTE      ADCCSTAT
*SFR* 000000B6H   DATA     WORD      ADCDR
*SFR* 000000B6H   DATA     BYTE      ADCDR0
*SFR* 000000B7H   DATA     BYTE      ADCDR1
*SFR* 000000ACH   DATA     BYTE      ADCGCR0
*SFR* 000000ADH   DATA     BYTE      ADCGCR1
*SFR* 000000B4H   DATA     BYTE      ADCGCR2
*SFR* 000000B5H   DATA     BYTE      ADCGCR3
*SFR* 000000F5H   DATA     BYTE      ADCHL
*SFR* 00000093H   DATA     BYTE      ADCIER
*SFR* 000000F7H   DATA     BYTE      ADCSPW
*SFR* 000000FDH   DATA     BYTE      ADCVREF
*SFR* 000000F0H   DATA     BYTE      B
*SFR* 000000F0H.0 DATA     BIT       B0
*SFR* 000000F0H.1 DATA     BIT       B1
*SFR* 000000F0H.2 DATA     BIT       B2
*SFR* 000000F0H.3 DATA     BIT       B3
*SFR* 000000F0H.4 DATA     BIT       B4
*SFR* 000000F0H.5 DATA     BIT       B5
*SFR* 000000F0H.6 DATA     BIT       B6
*SFR* 000000F0H.7 DATA     BIT       B7
*SFR* 00000086H   DATA     BYTE      BEEPCTR
*SFR* 000000F8H   DATA     BYTE      CLKCON
*SFR* 000000B1H   DATA     BYTE      CLKST
*SFR* 000000D0H.7 DATA     BIT       CY
*SFR* 00000083H   DATA     BYTE      DPH
*SFR* 00000085H   DATA     BYTE      DPH1
*SFR* 00000082H   DATA     BYTE      DPL
*SFR* 00000084H   DATA     BYTE      DPL1
*SFR* 00000092H   DATA     BYTE      DPS
*SFR* 000000A8H.7 DATA     BIT       EA
LX51 LINKER/LOCATER V4.66.97.0                                                        03/28/2025  17:08:22  PAGE 7


*SFR* 000000A8H.6 DATA     BIT       EADC
*SFR* 000000B8H.3 DATA     BIT       EFCINTEN
      01000B78H   CODE     ---       eflash_sn_test
      01000DA0H   CODE     ---       eflash_test
*SFR* 000000A8H.5 DATA     BIT       EPWM
*SFR* 000000D8H.3 DATA     BIT       ERSTF
*SFR* 000000A8H.4 DATA     BIT       ES0
*SFR* 000000A8H.2 DATA     BIT       ES1
*SFR* 000000B2H   DATA     BYTE      ESTCR
*SFR* 000000A8H.1 DATA     BIT       ET0
*SFR* 000000A8H.3 DATA     BIT       ET1
*SFR* 0000009EH   DATA     BYTE      EUARTEN
*SFR* 000000A8H.0 DATA     BIT       EX0
*SFR* 000000D0H.5 DATA     BIT       F0
*SFR* 000000D0H.1 DATA     BIT       F1
*SFR* 000000B8H.0 DATA     BIT       GTIM0INTEN
*SFR* 000000B8H.2 DATA     BIT       GTIM1INTEN
*SFR* 000000B8H.6 DATA     BIT       GTIM2INTEN
*SFR* 000000B8H.5 DATA     BIT       I2CINTEN
*SFR* 000000A8H   DATA     BYTE      IEN0
*SFR* 000000B8H   DATA     BYTE      IEN1
*SFR* 0000009AH   DATA     BYTE      IEN2
*SFR* 000000A9H   DATA     BYTE      IP0
*SFR* 000000B9H   DATA     BYTE      IP1
*SFR* 000000BDH   DATA     BYTE      LDOTRIMH
*SFR* 00000091H   DATA     BYTE      LDOTRIML
*SFR* 000000B8H.4 DATA     BIT       LPTIMINTEN
*SFR* 000000DDH   DATA     BYTE      LVDCON
*SFR* 000000D8H.5 DATA     BIT       LVRF
      01001135H   CODE     ---       main
*SFR* 000000D1H   DATA     WORD      OADR
*SFR* 000000D2H   DATA     BYTE      OADRH
*SFR* 000000D1H   DATA     BYTE      OADRL
*SFR* 000000D4H   DATA     BYTE      OCTRL
*SFR* 000000D3H   DATA     BYTE      ODATA
*SFR* 000000A2H   DATA     BYTE      OINTEN
*SFR* 000000A3H   DATA     BYTE      OINTUS
*SFR* 000000A7H   DATA     BYTE      OPSET
*SFR* 000000A5H   DATA     BYTE      OSEC
*SFR* 000000A6H   DATA     BYTE      OSTATUS
*SFR* 000000A1H   DATA     BYTE      OUS
*SFR* 000000D0H.0 DATA     BIT       P
*SFR* 00000080H   DATA     BYTE      P0
*SFR* 00000080H.0 DATA     BIT       P00
*SFR* 00000080H.1 DATA     BIT       P01
*SFR* 00000080H.2 DATA     BIT       P02
*SFR* 00000080H.3 DATA     BIT       P03
*SFR* 00000080H.4 DATA     BIT       P04
*SFR* 00000080H.5 DATA     BIT       P05
*SFR* 000000ABH   DATA     BYTE      P0AH
*SFR* 000000A4H   DATA     BYTE      P0AL
*SFR* 000000D7H   DATA     BYTE      P0CS
*SFR* 00000097H   DATA     BYTE      P0DR
*SFR* 000000E9H   DATA     BYTE      P0IEN
*SFR* 000000E1H   DATA     BYTE      P0IRQ
*SFR* 000000D6H   DATA     BYTE      P0OD
*SFR* 000000F9H   DATA     BYTE      P0OEN
*SFR* 000000D5H   DATA     BYTE      P0PD
*SFR* 000000F1H   DATA     BYTE      P0PU
*SFR* 00000090H   DATA     BYTE      P1
*SFR* 00000090H.0 DATA     BIT       P10
*SFR* 00000090H.1 DATA     BIT       P11
*SFR* 00000090H.2 DATA     BIT       P12
*SFR* 00000090H.3 DATA     BIT       P13
*SFR* 00000090H.4 DATA     BIT       P14
LX51 LINKER/LOCATER V4.66.97.0                                                        03/28/2025  17:08:22  PAGE 8


*SFR* 00000090H.5 DATA     BIT       P15
*SFR* 000000B0H   DATA     BYTE      P1AH
*SFR* 000000AEH   DATA     BYTE      P1AL
*SFR* 000000DCH   DATA     BYTE      P1CS
*SFR* 000000E5H   DATA     BYTE      P1DR
*SFR* 000000EAH   DATA     BYTE      P1IEN
*SFR* 000000E2H   DATA     BYTE      P1IRQ
*SFR* 000000DBH   DATA     BYTE      P1OD
*SFR* 000000FAH   DATA     BYTE      P1OEN
*SFR* 000000DAH   DATA     BYTE      P1PD
*SFR* 000000F2H   DATA     BYTE      P1PU
*SFR* 000000A0H   DATA     BYTE      P2
*SFR* 000000A0H.0 DATA     BIT       P20
*SFR* 000000A0H.2 DATA     BIT       P22
*SFR* 000000A0H.3 DATA     BIT       P23
*SFR* 000000A0H.5 DATA     BIT       P25
*SFR* 000000A0H.6 DATA     BIT       P26
*SFR* 000000A0H.7 DATA     BIT       P27
*SFR* 000000E8H   DATA     BYTE      P2AH
*SFR* 000000C0H   DATA     BYTE      P2AL
*SFR* 000000F4H   DATA     BYTE      P2CS
*SFR* 000000FCH   DATA     BYTE      P2DR
*SFR* 000000EBH   DATA     BYTE      P2IEN
*SFR* 000000E3H   DATA     BYTE      P2IRQ
*SFR* 000000ECH   DATA     BYTE      P2OD
*SFR* 000000FBH   DATA     BYTE      P2OEN
*SFR* 000000E4H   DATA     BYTE      P2PD
*SFR* 000000F3H   DATA     BYTE      P2PU
*SFR* 000000DEH   DATA     BYTE      PCLK0
*SFR* 000000DFH   DATA     BYTE      PCLK1
*SFR* 00000087H   DATA     BYTE      PCON
*SFR* 0000008EH   DATA     BYTE      PDSEL
*SFR* 0000008FH   DATA     BYTE      POREN
*SFR* 000000D8H.4 DATA     BIT       PORF
*SFR* 000000E6H   DATA     BYTE      PRESET0
*SFR* 000000E7H   DATA     BYTE      PRESET1
*SFR* 000000D0H   DATA     BYTE      PSW
*SFR* 000000C8H   DATA     BYTE      PWM0CON
*SFR* 000000C4H   DATA     BYTE      PWM0DH
*SFR* 000000C3H   DATA     BYTE      PWM0DL
*SFR* 000000C8H.7 DATA     BIT       PWM0EN
*SFR* 000000C8H.2 DATA     BIT       PWM0IE
*SFR* 000000C8H.1 DATA     BIT       PWM0IF
*SFR* 000000CCH   DATA     BYTE      PWM0PH
*SFR* 000000CBH   DATA     BYTE      PWM0PL
*SFR* 000000C8H.6 DATA     BIT       PWM0S
*SFR* 000000C8H.0 DATA     BIT       PWM0SS
*SFR* 000000C9H   DATA     BYTE      PWM1CON
*SFR* 000000C6H   DATA     BYTE      PWM1DH
*SFR* 000000C5H   DATA     BYTE      PWM1DL
*SFR* 000000CEH   DATA     BYTE      PWM1PH
*SFR* 000000CDH   DATA     BYTE      PWM1PL
*SFR* 000000CAH   DATA     BYTE      PWM2CON
*SFR* 000000C7H   DATA     BYTE      PWM2DH
*SFR* 000000CFH   DATA     BYTE      PWM2DL
*SFR* 000000C2H   DATA     BYTE      PWM2PH
*SFR* 000000C1H   DATA     BYTE      PWM2PL
*SFR* 00000098H.2 DATA     BIT       RB80
*SFR* 000000F8H.2 DATA     BIT       RC16MEN
*SFR* 000000F8H.5 DATA     BIT       RC16MF
*SFR* 000000F8H.3 DATA     BIT       RC32KEN
*SFR* 000000F8H.6 DATA     BIT       RC32KF
*SFR* 000000EEH   DATA     BYTE      RCHDIV
*SFR* 000000BEH   DATA     BYTE      RCHTRIMH
*SFR* 000000BFH   DATA     BYTE      RCHTRIML
LX51 LINKER/LOCATER V4.66.97.0                                                        03/28/2025  17:08:22  PAGE 9


      020000BCH   XDATA    DWORD     rchxxm
*SFR* 0000009FH   DATA     BYTE      RCLTRIMH
*SFR* 000000BCH   DATA     BYTE      RCLTRIML
      02000000H   XDATA    ---       read_data
*SFR* 000000AFH   DATA     BYTE      REMAP
*SFR* 00000098H.4 DATA     BIT       REN0
*SFR* 00000098H.0 DATA     BIT       RI0
*SFR* 000000D0H.3 DATA     BIT       RS0
*SFR* 000000D0H.4 DATA     BIT       RS1
*SFR* 000000D8H   DATA     BYTE      RSTSTAT
      02000069H   XDATA    WORD      rx_count
      02000068H   XDATA    BYTE      rx_flag
*SFR* 00000099H   DATA     BYTE      S0BUF
*SFR* 00000098H   DATA     BYTE      S0CON
*SFR* 000000BAH   DATA     BYTE      S0RELH
*SFR* 000000AAH   DATA     BYTE      S0RELL
*SFR* 0000009CH   DATA     BYTE      S1BUF
*SFR* 0000009BH   DATA     BYTE      S1CON
*SFR* 000000BBH   DATA     BYTE      S1RELH
*SFR* 0000009DH   DATA     BYTE      S1RELL
*SFR* 00000098H.7 DATA     BIT       SM0
*SFR* 00000098H.6 DATA     BIT       SM1
*SFR* 00000098H.5 DATA     BIT       SM20
*SFR* 00000081H   DATA     BYTE      SP
*SFR* 000000B8H.1 DATA     BIT       SPIINTEN
*SFR* 000000D9H   DATA     BYTE      SYSDIV
*SFR* 000000F8H.0 DATA     BIT       SYSSEL
      020000C0H   XDATA    DWORD     system_core_clock
      0100112AH   CODE     ---       system_init
*SFR* 00000098H.3 DATA     BIT       TB80
*SFR* 00000098H.1 DATA     BIT       TI0
      0200006BH   XDATA    WORD      tx_count
      020000C5H   XDATA    ---       uart0_func
      01000F85H   CODE     ---       UART0_IRQHandler
      010010E0H   CODE     ---       uart0_rec_pro
      01001148H   CODE     ---       uart0_recv_byte
      02000028H   XDATA    ---       uart0_rx_buf
      02000048H   XDATA    ---       uart0_tx_buf
      020000C4H   XDATA    BYTE      uart0_tx_flag
*SFR* 000000B8H.7 DATA     BIT       UART2INTEN
      01000003H   CODE     ---       uart_init
*SFR* 000000D8H.6 DATA     BIT       WDEN
*SFR* 000000D8H.7 DATA     BIT       WDOF
*SFR* 000000D8H.0 DATA     BIT       WDT0
*SFR* 000000D8H.1 DATA     BIT       WDT1
*SFR* 000000D8H.2 DATA     BIT       WDT2
      02000014H   XDATA    ---       write_data
*SFR* 000000F8H.1 DATA     BIT       XCLKEN
*SFR* 000000F8H.4 DATA     BIT       XCLKF
*SFR* 000000B3H   DATA     BYTE      XTHCTR



SYMBOL TABLE OF MODULE:  .\Out_Files\EFLASH_Example (?C_STARTUP)

      VALUE       REP       CLASS    TYPE      SYMBOL NAME
      ====================================================
      ---         MODULE    ---      ---       ?C_STARTUP
      01000000H   PUBLIC    CODE     ---       ?C_STARTUP
      000000E0H   SYMBOL    DATA     ---       ACC
      000000F0H   SYMBOL    DATA     ---       B
      00000083H   SYMBOL    DATA     ---       DPH
      00000082H   SYMBOL    DATA     ---       DPL
      00000000H   SYMBOL    NUMBER   ---       IBPSTACK
      00000100H   SYMBOL    NUMBER   ---       IBPSTACKTOP
LX51 LINKER/LOCATER V4.66.97.0                                                        03/28/2025  17:08:22  PAGE 10


      00000100H   SYMBOL    NUMBER   ---       IDATALEN
      01000C1AH   SYMBOL    CODE     ---       IDATALOOP
      00000000H   SYMBOL    NUMBER   ---       PBPSTACK
      00000100H   SYMBOL    NUMBER   ---       PBPSTACKTOP
      00000000H   SYMBOL    NUMBER   ---       PDATALEN
      00000000H   SYMBOL    NUMBER   ---       PDATASTART
      00000000H   SYMBOL    NUMBER   ---       PPAGE
      00000000H   SYMBOL    NUMBER   ---       PPAGEENABLE
      000000A0H   SYMBOL    DATA     ---       PPAGE_SFR
      00000081H   SYMBOL    DATA     ---       SP
      01000C17H   SYMBOL    CODE     ---       STARTUP1
      00000000H   SYMBOL    NUMBER   ---       XBPSTACK
      00000000H   SYMBOL    NUMBER   ---       XBPSTACKTOP
      00000800H   SYMBOL    NUMBER   ---       XDATALEN
      01000C25H   SYMBOL    CODE     ---       XDATALOOP
      00000000H   SYMBOL    NUMBER   ---       XDATASTART
      01000000H   LINE      CODE     ---       #126
      01000C17H   LINE      CODE     ---       #134
      01000C19H   LINE      CODE     ---       #135
      01000C1AH   LINE      CODE     ---       #136
      01000C1BH   LINE      CODE     ---       #137
      01000C1DH   LINE      CODE     ---       #142
      01000C20H   LINE      CODE     ---       #143
      01000C22H   LINE      CODE     ---       #147
      01000C24H   LINE      CODE     ---       #149
      01000C25H   LINE      CODE     ---       #150
      01000C26H   LINE      CODE     ---       #151
      01000C27H   LINE      CODE     ---       #152
      01000C29H   LINE      CODE     ---       #153
      01000C2BH   LINE      CODE     ---       #191
      01000C2EH   LINE      CODE     ---       #205

      ---         MODULE    ---      ---       SYSTEM_UM800XX
      020000C0H   PUBLIC    XDATA    DWORD     system_core_clock
      020000BCH   PUBLIC    XDATA    DWORD     rchxxm
      0100112AH   PUBLIC    CODE     ---       system_init
      010008C1H   PUBLIC    CODE     ---       _clock_init
      00000098H.3 SFRSYM    DATA     BIT       TB80
      000000E0H.7 SFRSYM    DATA     BIT       ACC7
      00000080H   SFRSYM    DATA     BYTE      P0
      00000090H   SFRSYM    DATA     BYTE      P1
      000000A0H   SFRSYM    DATA     BYTE      P2
      00000098H.5 SFRSYM    DATA     BIT       SM20
      000000B2H   SFRSYM    DATA     BYTE      ESTCR
      000000B1H   SFRSYM    DATA     BYTE      CLKST
      000000D0H.6 SFRSYM    DATA     BIT       AC
      000000D8H.3 SFRSYM    DATA     BIT       ERSTF
      000000E6H   SFRSYM    DATA     BYTE      PRESET0
      000000D4H   SFRSYM    DATA     BYTE      OCTRL
      000000A8H.7 SFRSYM    DATA     BIT       EA
      0000008FH   SFRSYM    DATA     BYTE      POREN
      000000C8H   SFRSYM    DATA     BYTE      PWM0CON
      000000E7H   SFRSYM    DATA     BYTE      PRESET1
      000000C9H   SFRSYM    DATA     BYTE      PWM1CON
      00000086H   SFRSYM    DATA     BYTE      BEEPCTR
      000000CAH   SFRSYM    DATA     BYTE      PWM2CON
      000000B8H.4 SFRSYM    DATA     BIT       LPTIMINTEN
      000000ABH   SFRSYM    DATA     BYTE      P0AH
      000000B0H   SFRSYM    DATA     BYTE      P1AH
      000000E8H   SFRSYM    DATA     BYTE      P2AH
      000000F8H.6 SFRSYM    DATA     BIT       RC32KF
      000000A8H   SFRSYM    DATA     BYTE      IEN0
      000000A7H   SFRSYM    DATA     BYTE      OPSET
      000000A4H   SFRSYM    DATA     BYTE      P0AL
      000000B8H   SFRSYM    DATA     BYTE      IEN1
LX51 LINKER/LOCATER V4.66.97.0                                                        03/28/2025  17:08:22  PAGE 11


      000000A8H.6 SFRSYM    DATA     BIT       EADC
      00000085H   SFRSYM    DATA     BYTE      DPH1
      000000AEH   SFRSYM    DATA     BYTE      P1AL
      0000009AH   SFRSYM    DATA     BYTE      IEN2
      000000C0H   SFRSYM    DATA     BYTE      P2AL
      000000B6H   SFRSYM    DATA     BYTE      ADCDR0
      000000F8H.5 SFRSYM    DATA     BIT       RC16MF
      000000B7H   SFRSYM    DATA     BYTE      ADCDR1
      00000084H   SFRSYM    DATA     BYTE      DPL1
      000000D6H   SFRSYM    DATA     BYTE      P0OD
      000000DBH   SFRSYM    DATA     BYTE      P1OD
      000000D5H   SFRSYM    DATA     BYTE      P0PD
      00000098H.4 SFRSYM    DATA     BIT       REN0
      000000ECH   SFRSYM    DATA     BYTE      P2OD
      000000DAH   SFRSYM    DATA     BYTE      P1PD
      000000E4H   SFRSYM    DATA     BYTE      P2PD
      000000D7H   SFRSYM    DATA     BYTE      P0CS
      00000097H   SFRSYM    DATA     BYTE      P0DR
      0000009EH   SFRSYM    DATA     BYTE      EUARTEN
      000000DCH   SFRSYM    DATA     BYTE      P1CS
      000000E5H   SFRSYM    DATA     BYTE      P1DR
      000000F4H   SFRSYM    DATA     BYTE      P2CS
      000000FCH   SFRSYM    DATA     BYTE      P2DR
      000000D0H.7 SFRSYM    DATA     BIT       CY
      000000D8H.0 SFRSYM    DATA     BIT       WDT0
      000000D8H.1 SFRSYM    DATA     BIT       WDT1
      000000D8H.2 SFRSYM    DATA     BIT       WDT2
      00000081H   SFRSYM    DATA     BYTE      SP
      000000F1H   SFRSYM    DATA     BYTE      P0PU
      000000F2H   SFRSYM    DATA     BYTE      P1PU
      000000D1H   SFRSYM    DATA     WORD      OADR
      000000F3H   SFRSYM    DATA     BYTE      P2PU
      00000093H   SFRSYM    DATA     BYTE      ADCIER
      000000A5H   SFRSYM    DATA     BYTE      OSEC
      000000D8H.6 SFRSYM    DATA     BIT       WDEN
      000000BAH   SFRSYM    DATA     BYTE      S0RELH
      00000080H.0 SFRSYM    DATA     BIT       P00
      000000D8H.7 SFRSYM    DATA     BIT       WDOF
      000000BBH   SFRSYM    DATA     BYTE      S1RELH
      00000090H.0 SFRSYM    DATA     BIT       P10
      00000080H.1 SFRSYM    DATA     BIT       P01
      00000087H   SFRSYM    DATA     BYTE      PCON
      000000C4H   SFRSYM    DATA     BYTE      PWM0DH
      000000A0H.0 SFRSYM    DATA     BIT       P20
      00000090H.1 SFRSYM    DATA     BIT       P11
      00000080H.2 SFRSYM    DATA     BIT       P02
      000000C6H   SFRSYM    DATA     BYTE      PWM1DH
      00000090H.2 SFRSYM    DATA     BIT       P12
      00000080H.3 SFRSYM    DATA     BIT       P03
      000000C7H   SFRSYM    DATA     BYTE      PWM2DH
      000000C8H.2 SFRSYM    DATA     BIT       PWM0IE
      000000AAH   SFRSYM    DATA     BYTE      S0RELL
      000000A0H.2 SFRSYM    DATA     BIT       P22
      00000090H.3 SFRSYM    DATA     BIT       P13
      00000080H.4 SFRSYM    DATA     BIT       P04
      000000C8H.1 SFRSYM    DATA     BIT       PWM0IF
      0000009DH   SFRSYM    DATA     BYTE      S1RELL
      000000A0H.3 SFRSYM    DATA     BIT       P23
      00000090H.4 SFRSYM    DATA     BIT       P14
      00000080H.5 SFRSYM    DATA     BIT       P05
      000000C3H   SFRSYM    DATA     BYTE      PWM0DL
      00000090H.5 SFRSYM    DATA     BIT       P15
      000000A6H   SFRSYM    DATA     BYTE      OSTATUS
      000000C5H   SFRSYM    DATA     BYTE      PWM1DL
      000000A0H.5 SFRSYM    DATA     BIT       P25
LX51 LINKER/LOCATER V4.66.97.0                                                        03/28/2025  17:08:22  PAGE 12


      000000D8H.4 SFRSYM    DATA     BIT       PORF
      000000D8H   SFRSYM    DATA     BYTE      RSTSTAT
      000000CFH   SFRSYM    DATA     BYTE      PWM2DL
      000000A0H.6 SFRSYM    DATA     BIT       P26
      000000C8H.7 SFRSYM    DATA     BIT       PWM0EN
      000000A0H.7 SFRSYM    DATA     BIT       P27
      000000A8H.5 SFRSYM    DATA     BIT       EPWM
      000000D8H.5 SFRSYM    DATA     BIT       LVRF
      000000F8H   SFRSYM    DATA     BYTE      CLKCON
      000000CCH   SFRSYM    DATA     BYTE      PWM0PH
      000000CEH   SFRSYM    DATA     BYTE      PWM1PH
      000000B8H.5 SFRSYM    DATA     BIT       I2CINTEN
      000000C2H   SFRSYM    DATA     BYTE      PWM2PH
      000000F0H   SFRSYM    DATA     BYTE      B
      000000EEH   SFRSYM    DATA     BYTE      RCHDIV
      000000CBH   SFRSYM    DATA     BYTE      PWM0PL
      000000CDH   SFRSYM    DATA     BYTE      PWM1PL
      000000C1H   SFRSYM    DATA     BYTE      PWM2PL
      000000F7H   SFRSYM    DATA     BYTE      ADCSPW
      000000F8H.1 SFRSYM    DATA     BIT       XCLKEN
      000000E0H   SFRSYM    DATA     BYTE      ACC
      000000DDH   SFRSYM    DATA     BYTE      LVDCON
      000000A8H.4 SFRSYM    DATA     BIT       ES0
      000000A9H   SFRSYM    DATA     BYTE      IP0
      000000A8H.1 SFRSYM    DATA     BIT       ET0
      000000A8H.2 SFRSYM    DATA     BIT       ES1
      000000F6H   SFRSYM    DATA     BYTE      ADCCSTAT
      000000B9H   SFRSYM    DATA     BYTE      IP1
      000000A8H.3 SFRSYM    DATA     BIT       ET1
      00000098H.0 SFRSYM    DATA     BIT       RI0
      000000C8H.0 SFRSYM    DATA     BIT       PWM0SS
      00000098H.1 SFRSYM    DATA     BIT       TI0
      000000A8H.0 SFRSYM    DATA     BIT       EX0
      000000D0H.0 SFRSYM    DATA     BIT       P
      000000B8H.3 SFRSYM    DATA     BIT       EFCINTEN
      000000A2H   SFRSYM    DATA     BYTE      OINTEN
      00000098H.7 SFRSYM    DATA     BIT       SM0
      00000098H.6 SFRSYM    DATA     BIT       SM1
      000000FEH   SFRSYM    DATA     BYTE      ADCCDR0
      000000FFH   SFRSYM    DATA     BYTE      ADCCDR1
      000000D0H.3 SFRSYM    DATA     BIT       RS0
      000000ACH   SFRSYM    DATA     BYTE      ADCGCR0
      000000D0H.4 SFRSYM    DATA     BIT       RS1
      000000ADH   SFRSYM    DATA     BYTE      ADCGCR1
      000000B4H   SFRSYM    DATA     BYTE      ADCGCR2
      000000B5H   SFRSYM    DATA     BYTE      ADCGCR3
      000000F8H.3 SFRSYM    DATA     BIT       RC32KEN
      000000DEH   SFRSYM    DATA     BYTE      PCLK0
      000000DFH   SFRSYM    DATA     BYTE      PCLK1
      00000083H   SFRSYM    DATA     BYTE      DPH
      000000E9H   SFRSYM    DATA     BYTE      P0IEN
      000000F5H   SFRSYM    DATA     BYTE      ADCHL
      000000F8H.2 SFRSYM    DATA     BIT       RC16MEN
      000000EAH   SFRSYM    DATA     BYTE      P1IEN
      000000EBH   SFRSYM    DATA     BYTE      P2IEN
      000000B6H   SFRSYM    DATA     WORD      ADCDR
      000000B3H   SFRSYM    DATA     BYTE      XTHCTR
      00000082H   SFRSYM    DATA     BYTE      DPL
      00000099H   SFRSYM    DATA     BYTE      S0BUF
      0000009CH   SFRSYM    DATA     BYTE      S1BUF
      000000F9H   SFRSYM    DATA     BYTE      P0OEN
      000000B8H.0 SFRSYM    DATA     BIT       GTIM0INTEN
      000000D9H   SFRSYM    DATA     BYTE      SYSDIV
      00000098H   SFRSYM    DATA     BYTE      S0CON
      000000FAH   SFRSYM    DATA     BYTE      P1OEN
LX51 LINKER/LOCATER V4.66.97.0                                                        03/28/2025  17:08:22  PAGE 13


      000000B8H.2 SFRSYM    DATA     BIT       GTIM1INTEN
      000000A3H   SFRSYM    DATA     BYTE      OINTUS
      000000BEH   SFRSYM    DATA     BYTE      RCHTRIMH
      000000F8H.0 SFRSYM    DATA     BIT       SYSSEL
      0000009BH   SFRSYM    DATA     BYTE      S1CON
      000000FBH   SFRSYM    DATA     BYTE      P2OEN
      000000B8H.6 SFRSYM    DATA     BIT       GTIM2INTEN
      000000BDH   SFRSYM    DATA     BYTE      LDOTRIMH
      00000092H   SFRSYM    DATA     BYTE      DPS
      0000009FH   SFRSYM    DATA     BYTE      RCLTRIMH
      000000BFH   SFRSYM    DATA     BYTE      RCHTRIML
      000000D3H   SFRSYM    DATA     BYTE      ODATA
      00000091H   SFRSYM    DATA     BYTE      LDOTRIML
      000000BCH   SFRSYM    DATA     BYTE      RCLTRIML
      000000E1H   SFRSYM    DATA     BYTE      P0IRQ
      000000B8H.1 SFRSYM    DATA     BIT       SPIINTEN
      000000E2H   SFRSYM    DATA     BYTE      P1IRQ
      000000E3H   SFRSYM    DATA     BYTE      P2IRQ
      000000D2H   SFRSYM    DATA     BYTE      OADRH
      000000B8H.7 SFRSYM    DATA     BIT       UART2INTEN
      000000F0H.0 SFRSYM    DATA     BIT       B0
      000000F0H.1 SFRSYM    DATA     BIT       B1
      000000F0H.2 SFRSYM    DATA     BIT       B2
      000000D1H   SFRSYM    DATA     BYTE      OADRL
      000000F0H.3 SFRSYM    DATA     BIT       B3
      000000F0H.4 SFRSYM    DATA     BIT       B4
      000000D0H.5 SFRSYM    DATA     BIT       F0
      000000F0H.5 SFRSYM    DATA     BIT       B5
      000000D0H.1 SFRSYM    DATA     BIT       F1
      000000AFH   SFRSYM    DATA     BYTE      REMAP
      000000F0H.6 SFRSYM    DATA     BIT       B6
      000000E0H.0 SFRSYM    DATA     BIT       ACC0
      000000A1H   SFRSYM    DATA     BYTE      OUS
      000000C8H.6 SFRSYM    DATA     BIT       PWM0S
      000000F0H.7 SFRSYM    DATA     BIT       B7
      000000E0H.1 SFRSYM    DATA     BIT       ACC1
      000000F8H.4 SFRSYM    DATA     BIT       XCLKF
      000000E0H.2 SFRSYM    DATA     BIT       ACC2
      0000008EH   SFRSYM    DATA     BYTE      PDSEL
      000000E0H.3 SFRSYM    DATA     BIT       ACC3
      000000D0H   SFRSYM    DATA     BYTE      PSW
      000000E0H.4 SFRSYM    DATA     BIT       ACC4
      00000098H.2 SFRSYM    DATA     BIT       RB80
      000000E0H.5 SFRSYM    DATA     BIT       ACC5
      000000FDH   SFRSYM    DATA     BYTE      ADCVREF
      000000E0H.6 SFRSYM    DATA     BIT       ACC6

      010008C1H   BLOCK     CODE     ---       LVL=0
      0200006DH   SYMBOL    XDATA    DWORD     system_clk_hz
      010008C7H   BLOCK     CODE     NEAR LAB  LVL=1
      02000071H   SYMBOL    XDATA    DWORD     crystal_clk
      ---         BLOCKEND  ---      ---       LVL=1
      010008C1H   LINE      CODE     ---       #25
      010008C7H   LINE      CODE     ---       #26
      010008C7H   LINE      CODE     ---       #27
      010008D1H   LINE      CODE     ---       #29
      010008D4H   LINE      CODE     ---       #30
      010008DCH   LINE      CODE     ---       #34
      01000944H   LINE      CODE     ---       #40
      0100096CH   LINE      CODE     ---       #41
      0100096CH   LINE      CODE     ---       #42
      0100096CH   LINE      CODE     ---       #43
      0100096EH   LINE      CODE     ---       #44
      01000980H   LINE      CODE     ---       #45
      01000980H   LINE      CODE     ---       #46
LX51 LINKER/LOCATER V4.66.97.0                                                        03/28/2025  17:08:22  PAGE 14


      0100098AH   LINE      CODE     ---       #47
      0100098CH   LINE      CODE     ---       #49
      0100098CH   LINE      CODE     ---       #50
      010009A1H   LINE      CODE     ---       #51
      010009A1H   LINE      CODE     ---       #53
      010009C6H   LINE      CODE     ---       #54
      010009C6H   LINE      CODE     ---       #55
      010009C6H   LINE      CODE     ---       #56
      010009C9H   LINE      CODE     ---       #57
      010009C9H   LINE      CODE     ---       #58
      010009C9H   LINE      CODE     ---       #59
      010009CBH   LINE      CODE     ---       #61
      010009CBH   LINE      CODE     ---       #62
      010009CEH   LINE      CODE     ---       #63
      010009CEH   LINE      CODE     ---       #64
      010009CEH   LINE      CODE     ---       #65
      010009D0H   LINE      CODE     ---       #67
      010009D0H   LINE      CODE     ---       #68
      010009D3H   LINE      CODE     ---       #69
      010009D6H   LINE      CODE     ---       #70
      010009D6H   LINE      CODE     ---       #71
      010009D8H   LINE      CODE     ---       #73
      010009D8H   LINE      CODE     ---       #74
      010009DBH   LINE      CODE     ---       #75
      010009DEH   LINE      CODE     ---       #76
      010009E4H   LINE      CODE     ---       #77
      010009E6H   LINE      CODE     ---       #79
      010009E6H   LINE      CODE     ---       #80
      010009E9H   LINE      CODE     ---       #81
      010009ECH   LINE      CODE     ---       #82
      01000A00H   LINE      CODE     ---       #83
      01000A00H   LINE      CODE     ---       #84
      01000A00H   LINE      CODE     ---       #120
      01000A03H   LINE      CODE     ---       #121
      ---         BLOCKEND  ---      ---       LVL=0

      0100112AH   BLOCK     CODE     ---       LVL=0
      0100112AH   LINE      CODE     ---       #130
      0100112AH   LINE      CODE     ---       #131
      0100112AH   LINE      CODE     ---       #132
      ---         BLOCKEND  ---      ---       LVL=0

      ---         MODULE    ---      ---       COMMON
      01000E0DH   PUBLIC    CODE     ---       _printf_buff_byte
      01000FCFH   PUBLIC    CODE     ---       _delay1ms
      00000098H.3 SFRSYM    DATA     BIT       TB80
      000000E0H.7 SFRSYM    DATA     BIT       ACC7
      00000080H   SFRSYM    DATA     BYTE      P0
      00000090H   SFRSYM    DATA     BYTE      P1
      000000A0H   SFRSYM    DATA     BYTE      P2
      00000098H.5 SFRSYM    DATA     BIT       SM20
      000000B2H   SFRSYM    DATA     BYTE      ESTCR
      000000B1H   SFRSYM    DATA     BYTE      CLKST
      000000D0H.6 SFRSYM    DATA     BIT       AC
      000000D8H.3 SFRSYM    DATA     BIT       ERSTF
      000000E6H   SFRSYM    DATA     BYTE      PRESET0
      000000D4H   SFRSYM    DATA     BYTE      OCTRL
      000000A8H.7 SFRSYM    DATA     BIT       EA
      0000008FH   SFRSYM    DATA     BYTE      POREN
      000000C8H   SFRSYM    DATA     BYTE      PWM0CON
      000000E7H   SFRSYM    DATA     BYTE      PRESET1
      000000C9H   SFRSYM    DATA     BYTE      PWM1CON
      00000086H   SFRSYM    DATA     BYTE      BEEPCTR
      000000CAH   SFRSYM    DATA     BYTE      PWM2CON
      000000B8H.4 SFRSYM    DATA     BIT       LPTIMINTEN
LX51 LINKER/LOCATER V4.66.97.0                                                        03/28/2025  17:08:22  PAGE 15


      000000ABH   SFRSYM    DATA     BYTE      P0AH
      000000B0H   SFRSYM    DATA     BYTE      P1AH
      000000E8H   SFRSYM    DATA     BYTE      P2AH
      000000F8H.6 SFRSYM    DATA     BIT       RC32KF
      000000A8H   SFRSYM    DATA     BYTE      IEN0
      000000A7H   SFRSYM    DATA     BYTE      OPSET
      000000A4H   SFRSYM    DATA     BYTE      P0AL
      000000B8H   SFRSYM    DATA     BYTE      IEN1
      000000A8H.6 SFRSYM    DATA     BIT       EADC
      00000085H   SFRSYM    DATA     BYTE      DPH1
      000000AEH   SFRSYM    DATA     BYTE      P1AL
      0000009AH   SFRSYM    DATA     BYTE      IEN2
      000000C0H   SFRSYM    DATA     BYTE      P2AL
      000000B6H   SFRSYM    DATA     BYTE      ADCDR0
      000000F8H.5 SFRSYM    DATA     BIT       RC16MF
      000000B7H   SFRSYM    DATA     BYTE      ADCDR1
      00000084H   SFRSYM    DATA     BYTE      DPL1
      000000D6H   SFRSYM    DATA     BYTE      P0OD
      000000DBH   SFRSYM    DATA     BYTE      P1OD
      000000D5H   SFRSYM    DATA     BYTE      P0PD
      00000098H.4 SFRSYM    DATA     BIT       REN0
      000000ECH   SFRSYM    DATA     BYTE      P2OD
      000000DAH   SFRSYM    DATA     BYTE      P1PD
      000000E4H   SFRSYM    DATA     BYTE      P2PD
      000000D7H   SFRSYM    DATA     BYTE      P0CS
      00000097H   SFRSYM    DATA     BYTE      P0DR
      0000009EH   SFRSYM    DATA     BYTE      EUARTEN
      000000DCH   SFRSYM    DATA     BYTE      P1CS
      000000E5H   SFRSYM    DATA     BYTE      P1DR
      000000F4H   SFRSYM    DATA     BYTE      P2CS
      000000FCH   SFRSYM    DATA     BYTE      P2DR
      000000D0H.7 SFRSYM    DATA     BIT       CY
      000000D8H.0 SFRSYM    DATA     BIT       WDT0
      000000D8H.1 SFRSYM    DATA     BIT       WDT1
      000000D8H.2 SFRSYM    DATA     BIT       WDT2
      00000081H   SFRSYM    DATA     BYTE      SP
      000000F1H   SFRSYM    DATA     BYTE      P0PU
      000000F2H   SFRSYM    DATA     BYTE      P1PU
      000000D1H   SFRSYM    DATA     WORD      OADR
      000000F3H   SFRSYM    DATA     BYTE      P2PU
      00000093H   SFRSYM    DATA     BYTE      ADCIER
      000000A5H   SFRSYM    DATA     BYTE      OSEC
      000000D8H.6 SFRSYM    DATA     BIT       WDEN
      000000BAH   SFRSYM    DATA     BYTE      S0RELH
      00000080H.0 SFRSYM    DATA     BIT       P00
      000000D8H.7 SFRSYM    DATA     BIT       WDOF
      000000BBH   SFRSYM    DATA     BYTE      S1RELH
      00000090H.0 SFRSYM    DATA     BIT       P10
      00000080H.1 SFRSYM    DATA     BIT       P01
      00000087H   SFRSYM    DATA     BYTE      PCON
      000000C4H   SFRSYM    DATA     BYTE      PWM0DH
      000000A0H.0 SFRSYM    DATA     BIT       P20
      00000090H.1 SFRSYM    DATA     BIT       P11
      00000080H.2 SFRSYM    DATA     BIT       P02
      000000C6H   SFRSYM    DATA     BYTE      PWM1DH
      00000090H.2 SFRSYM    DATA     BIT       P12
      00000080H.3 SFRSYM    DATA     BIT       P03
      000000C7H   SFRSYM    DATA     BYTE      PWM2DH
      000000C8H.2 SFRSYM    DATA     BIT       PWM0IE
      000000AAH   SFRSYM    DATA     BYTE      S0RELL
      000000A0H.2 SFRSYM    DATA     BIT       P22
      00000090H.3 SFRSYM    DATA     BIT       P13
      00000080H.4 SFRSYM    DATA     BIT       P04
      000000C8H.1 SFRSYM    DATA     BIT       PWM0IF
      0000009DH   SFRSYM    DATA     BYTE      S1RELL
LX51 LINKER/LOCATER V4.66.97.0                                                        03/28/2025  17:08:22  PAGE 16


      000000A0H.3 SFRSYM    DATA     BIT       P23
      00000090H.4 SFRSYM    DATA     BIT       P14
      00000080H.5 SFRSYM    DATA     BIT       P05
      000000C3H   SFRSYM    DATA     BYTE      PWM0DL
      00000090H.5 SFRSYM    DATA     BIT       P15
      000000A6H   SFRSYM    DATA     BYTE      OSTATUS
      000000C5H   SFRSYM    DATA     BYTE      PWM1DL
      000000A0H.5 SFRSYM    DATA     BIT       P25
      000000D8H.4 SFRSYM    DATA     BIT       PORF
      000000D8H   SFRSYM    DATA     BYTE      RSTSTAT
      000000CFH   SFRSYM    DATA     BYTE      PWM2DL
      000000A0H.6 SFRSYM    DATA     BIT       P26
      000000C8H.7 SFRSYM    DATA     BIT       PWM0EN
      000000A0H.7 SFRSYM    DATA     BIT       P27
      000000A8H.5 SFRSYM    DATA     BIT       EPWM
      000000D8H.5 SFRSYM    DATA     BIT       LVRF
      000000F8H   SFRSYM    DATA     BYTE      CLKCON
      000000CCH   SFRSYM    DATA     BYTE      PWM0PH
      000000CEH   SFRSYM    DATA     BYTE      PWM1PH
      000000B8H.5 SFRSYM    DATA     BIT       I2CINTEN
      000000C2H   SFRSYM    DATA     BYTE      PWM2PH
      000000F0H   SFRSYM    DATA     BYTE      B
      000000EEH   SFRSYM    DATA     BYTE      RCHDIV
      000000CBH   SFRSYM    DATA     BYTE      PWM0PL
      000000CDH   SFRSYM    DATA     BYTE      PWM1PL
      000000C1H   SFRSYM    DATA     BYTE      PWM2PL
      000000F7H   SFRSYM    DATA     BYTE      ADCSPW
      000000F8H.1 SFRSYM    DATA     BIT       XCLKEN
      000000E0H   SFRSYM    DATA     BYTE      ACC
      000000DDH   SFRSYM    DATA     BYTE      LVDCON
      000000A8H.4 SFRSYM    DATA     BIT       ES0
      000000A9H   SFRSYM    DATA     BYTE      IP0
      000000A8H.1 SFRSYM    DATA     BIT       ET0
      000000A8H.2 SFRSYM    DATA     BIT       ES1
      000000F6H   SFRSYM    DATA     BYTE      ADCCSTAT
      000000B9H   SFRSYM    DATA     BYTE      IP1
      000000A8H.3 SFRSYM    DATA     BIT       ET1
      00000098H.0 SFRSYM    DATA     BIT       RI0
      000000C8H.0 SFRSYM    DATA     BIT       PWM0SS
      00000098H.1 SFRSYM    DATA     BIT       TI0
      000000A8H.0 SFRSYM    DATA     BIT       EX0
      000000D0H.0 SFRSYM    DATA     BIT       P
      000000B8H.3 SFRSYM    DATA     BIT       EFCINTEN
      000000A2H   SFRSYM    DATA     BYTE      OINTEN
      00000098H.7 SFRSYM    DATA     BIT       SM0
      00000098H.6 SFRSYM    DATA     BIT       SM1
      000000FEH   SFRSYM    DATA     BYTE      ADCCDR0
      000000FFH   SFRSYM    DATA     BYTE      ADCCDR1
      000000D0H.3 SFRSYM    DATA     BIT       RS0
      000000ACH   SFRSYM    DATA     BYTE      ADCGCR0
      000000D0H.4 SFRSYM    DATA     BIT       RS1
      000000ADH   SFRSYM    DATA     BYTE      ADCGCR1
      000000B4H   SFRSYM    DATA     BYTE      ADCGCR2
      000000B5H   SFRSYM    DATA     BYTE      ADCGCR3
      000000F8H.3 SFRSYM    DATA     BIT       RC32KEN
      000000DEH   SFRSYM    DATA     BYTE      PCLK0
      000000DFH   SFRSYM    DATA     BYTE      PCLK1
      00000083H   SFRSYM    DATA     BYTE      DPH
      000000E9H   SFRSYM    DATA     BYTE      P0IEN
      000000F5H   SFRSYM    DATA     BYTE      ADCHL
      000000F8H.2 SFRSYM    DATA     BIT       RC16MEN
      000000EAH   SFRSYM    DATA     BYTE      P1IEN
      000000EBH   SFRSYM    DATA     BYTE      P2IEN
      000000B6H   SFRSYM    DATA     WORD      ADCDR
      000000B3H   SFRSYM    DATA     BYTE      XTHCTR
LX51 LINKER/LOCATER V4.66.97.0                                                        03/28/2025  17:08:22  PAGE 17


      00000082H   SFRSYM    DATA     BYTE      DPL
      00000099H   SFRSYM    DATA     BYTE      S0BUF
      0000009CH   SFRSYM    DATA     BYTE      S1BUF
      000000F9H   SFRSYM    DATA     BYTE      P0OEN
      000000B8H.0 SFRSYM    DATA     BIT       GTIM0INTEN
      000000D9H   SFRSYM    DATA     BYTE      SYSDIV
      00000098H   SFRSYM    DATA     BYTE      S0CON
      000000FAH   SFRSYM    DATA     BYTE      P1OEN
      000000B8H.2 SFRSYM    DATA     BIT       GTIM1INTEN
      000000A3H   SFRSYM    DATA     BYTE      OINTUS
      000000BEH   SFRSYM    DATA     BYTE      RCHTRIMH
      000000F8H.0 SFRSYM    DATA     BIT       SYSSEL
      0000009BH   SFRSYM    DATA     BYTE      S1CON
      000000FBH   SFRSYM    DATA     BYTE      P2OEN
      000000B8H.6 SFRSYM    DATA     BIT       GTIM2INTEN
      000000BDH   SFRSYM    DATA     BYTE      LDOTRIMH
      00000092H   SFRSYM    DATA     BYTE      DPS
      0000009FH   SFRSYM    DATA     BYTE      RCLTRIMH
      000000BFH   SFRSYM    DATA     BYTE      RCHTRIML
      000000D3H   SFRSYM    DATA     BYTE      ODATA
      00000091H   SFRSYM    DATA     BYTE      LDOTRIML
      000000BCH   SFRSYM    DATA     BYTE      RCLTRIML
      000000E1H   SFRSYM    DATA     BYTE      P0IRQ
      000000B8H.1 SFRSYM    DATA     BIT       SPIINTEN
      000000E2H   SFRSYM    DATA     BYTE      P1IRQ
      000000E3H   SFRSYM    DATA     BYTE      P2IRQ
      000000D2H   SFRSYM    DATA     BYTE      OADRH
      000000B8H.7 SFRSYM    DATA     BIT       UART2INTEN
      000000F0H.0 SFRSYM    DATA     BIT       B0
      000000F0H.1 SFRSYM    DATA     BIT       B1
      000000F0H.2 SFRSYM    DATA     BIT       B2
      000000D1H   SFRSYM    DATA     BYTE      OADRL
      000000F0H.3 SFRSYM    DATA     BIT       B3
      000000F0H.4 SFRSYM    DATA     BIT       B4
      000000D0H.5 SFRSYM    DATA     BIT       F0
      000000F0H.5 SFRSYM    DATA     BIT       B5
      000000D0H.1 SFRSYM    DATA     BIT       F1
      000000AFH   SFRSYM    DATA     BYTE      REMAP
      000000F0H.6 SFRSYM    DATA     BIT       B6
      000000E0H.0 SFRSYM    DATA     BIT       ACC0
      000000A1H   SFRSYM    DATA     BYTE      OUS
      000000C8H.6 SFRSYM    DATA     BIT       PWM0S
      000000F0H.7 SFRSYM    DATA     BIT       B7
      000000E0H.1 SFRSYM    DATA     BIT       ACC1
      000000F8H.4 SFRSYM    DATA     BIT       XCLKF
      000000E0H.2 SFRSYM    DATA     BIT       ACC2
      0000008EH   SFRSYM    DATA     BYTE      PDSEL
      000000E0H.3 SFRSYM    DATA     BIT       ACC3
      000000D0H   SFRSYM    DATA     BYTE      PSW
      000000E0H.4 SFRSYM    DATA     BIT       ACC4
      00000098H.2 SFRSYM    DATA     BIT       RB80
      000000E0H.5 SFRSYM    DATA     BIT       ACC5
      000000FDH   SFRSYM    DATA     BYTE      ADCVREF
      000000E0H.6 SFRSYM    DATA     BIT       ACC6

      01000FCFH   BLOCK     CODE     ---       LVL=0
      0200006DH   SYMBOL    XDATA    DWORD     n
      01000FD5H   BLOCK     CODE     NEAR LAB  LVL=1
      02000071H   SYMBOL    XDATA    DWORD     x
      00000007H   SYMBOL    DATA     BYTE      i
      00000006H   SYMBOL    DATA     BYTE      j
      ---         BLOCKEND  ---      ---       LVL=1
      01000FCFH   LINE      CODE     ---       #20
      01000FD5H   LINE      CODE     ---       #21
      01000FD5H   LINE      CODE     ---       #25
LX51 LINKER/LOCATER V4.66.97.0                                                        03/28/2025  17:08:22  PAGE 18


      01000FF1H   LINE      CODE     ---       #26
      01000FF1H   LINE      CODE     ---       #27
      01000FF2H   LINE      CODE     ---       #28
      01000FF4H   LINE      CODE     ---       #29
      01000FF6H   LINE      CODE     ---       #31
      01000FF6H   LINE      CODE     ---       #32
      01000FF8H   LINE      CODE     ---       #33
      01000FFAH   LINE      CODE     ---       #34
      01001015H   LINE      CODE     ---       #35
      ---         BLOCKEND  ---      ---       LVL=0

      01000E0DH   BLOCK     CODE     ---       LVL=0
      02000089H   SYMBOL    XDATA    ---       buff
      0200008CH   SYMBOL    XDATA    DWORD     length
      01000E19H   BLOCK     CODE     NEAR LAB  LVL=1
      02000090H   SYMBOL    XDATA    DWORD     i
      ---         BLOCKEND  ---      ---       LVL=1
      01000E0DH   LINE      CODE     ---       #58
      01000E19H   LINE      CODE     ---       #59
      01000E19H   LINE      CODE     ---       #62
      01000E35H   LINE      CODE     ---       #63
      01000E35H   LINE      CODE     ---       #64
      01000E55H   LINE      CODE     ---       #65
      01000E70H   LINE      CODE     ---       #66
      ---         BLOCKEND  ---      ---       LVL=0

      ---         MODULE    ---      ---       EFLASH
      01000EDEH   PUBLIC    CODE     ---       _read_Vcap
      01000A04H   PUBLIC    CODE     ---       _read_UID
      01001081H   PUBLIC    CODE     ---       _read_sequence
      02000078H   PUBLIC    XDATA    BYTE      ?_eflash_read_bytes?BYTE
      01000CB1H   PUBLIC    CODE     ---       _eflash_read_bytes
      01001140H   PUBLIC    CODE     ---       _eflash_read_byte
      02000078H   PUBLIC    XDATA    BYTE      ?_eflash_write_bytes?BYTE
      01000E79H   PUBLIC    CODE     ---       _eflash_write_bytes
      010010B2H   PUBLIC    CODE     ---       _eflash_erase_page
      0100104DH   PUBLIC    CODE     ---       _eflash_init
      00000098H.3 SFRSYM    DATA     BIT       TB80
      000000E0H.7 SFRSYM    DATA     BIT       ACC7
      00000080H   SFRSYM    DATA     BYTE      P0
      00000090H   SFRSYM    DATA     BYTE      P1
      000000A0H   SFRSYM    DATA     BYTE      P2
      00000098H.5 SFRSYM    DATA     BIT       SM20
      000000B2H   SFRSYM    DATA     BYTE      ESTCR
      000000B1H   SFRSYM    DATA     BYTE      CLKST
      000000D0H.6 SFRSYM    DATA     BIT       AC
      000000D8H.3 SFRSYM    DATA     BIT       ERSTF
      000000E6H   SFRSYM    DATA     BYTE      PRESET0
      000000D4H   SFRSYM    DATA     BYTE      OCTRL
      000000A8H.7 SFRSYM    DATA     BIT       EA
      0000008FH   SFRSYM    DATA     BYTE      POREN
      000000C8H   SFRSYM    DATA     BYTE      PWM0CON
      000000E7H   SFRSYM    DATA     BYTE      PRESET1
      000000C9H   SFRSYM    DATA     BYTE      PWM1CON
      00000086H   SFRSYM    DATA     BYTE      BEEPCTR
      000000CAH   SFRSYM    DATA     BYTE      PWM2CON
      000000B8H.4 SFRSYM    DATA     BIT       LPTIMINTEN
      000000ABH   SFRSYM    DATA     BYTE      P0AH
      000000B0H   SFRSYM    DATA     BYTE      P1AH
      000000E8H   SFRSYM    DATA     BYTE      P2AH
      000000F8H.6 SFRSYM    DATA     BIT       RC32KF
      000000A8H   SFRSYM    DATA     BYTE      IEN0
      000000A7H   SFRSYM    DATA     BYTE      OPSET
      000000A4H   SFRSYM    DATA     BYTE      P0AL
      000000B8H   SFRSYM    DATA     BYTE      IEN1
LX51 LINKER/LOCATER V4.66.97.0                                                        03/28/2025  17:08:22  PAGE 19


      000000A8H.6 SFRSYM    DATA     BIT       EADC
      00000085H   SFRSYM    DATA     BYTE      DPH1
      000000AEH   SFRSYM    DATA     BYTE      P1AL
      0000009AH   SFRSYM    DATA     BYTE      IEN2
      000000C0H   SFRSYM    DATA     BYTE      P2AL
      000000B6H   SFRSYM    DATA     BYTE      ADCDR0
      000000F8H.5 SFRSYM    DATA     BIT       RC16MF
      000000B7H   SFRSYM    DATA     BYTE      ADCDR1
      00000084H   SFRSYM    DATA     BYTE      DPL1
      000000D6H   SFRSYM    DATA     BYTE      P0OD
      000000DBH   SFRSYM    DATA     BYTE      P1OD
      000000D5H   SFRSYM    DATA     BYTE      P0PD
      00000098H.4 SFRSYM    DATA     BIT       REN0
      000000ECH   SFRSYM    DATA     BYTE      P2OD
      000000DAH   SFRSYM    DATA     BYTE      P1PD
      000000E4H   SFRSYM    DATA     BYTE      P2PD
      000000D7H   SFRSYM    DATA     BYTE      P0CS
      00000097H   SFRSYM    DATA     BYTE      P0DR
      0000009EH   SFRSYM    DATA     BYTE      EUARTEN
      000000DCH   SFRSYM    DATA     BYTE      P1CS
      000000E5H   SFRSYM    DATA     BYTE      P1DR
      000000F4H   SFRSYM    DATA     BYTE      P2CS
      000000FCH   SFRSYM    DATA     BYTE      P2DR
      000000D0H.7 SFRSYM    DATA     BIT       CY
      000000D8H.0 SFRSYM    DATA     BIT       WDT0
      000000D8H.1 SFRSYM    DATA     BIT       WDT1
      000000D8H.2 SFRSYM    DATA     BIT       WDT2
      00000081H   SFRSYM    DATA     BYTE      SP
      000000F1H   SFRSYM    DATA     BYTE      P0PU
      000000F2H   SFRSYM    DATA     BYTE      P1PU
      000000D1H   SFRSYM    DATA     WORD      OADR
      000000F3H   SFRSYM    DATA     BYTE      P2PU
      00000093H   SFRSYM    DATA     BYTE      ADCIER
      000000A5H   SFRSYM    DATA     BYTE      OSEC
      000000D8H.6 SFRSYM    DATA     BIT       WDEN
      000000BAH   SFRSYM    DATA     BYTE      S0RELH
      00000080H.0 SFRSYM    DATA     BIT       P00
      000000D8H.7 SFRSYM    DATA     BIT       WDOF
      000000BBH   SFRSYM    DATA     BYTE      S1RELH
      00000090H.0 SFRSYM    DATA     BIT       P10
      00000080H.1 SFRSYM    DATA     BIT       P01
      00000087H   SFRSYM    DATA     BYTE      PCON
      000000C4H   SFRSYM    DATA     BYTE      PWM0DH
      000000A0H.0 SFRSYM    DATA     BIT       P20
      00000090H.1 SFRSYM    DATA     BIT       P11
      00000080H.2 SFRSYM    DATA     BIT       P02
      000000C6H   SFRSYM    DATA     BYTE      PWM1DH
      00000090H.2 SFRSYM    DATA     BIT       P12
      00000080H.3 SFRSYM    DATA     BIT       P03
      000000C7H   SFRSYM    DATA     BYTE      PWM2DH
      000000C8H.2 SFRSYM    DATA     BIT       PWM0IE
      000000AAH   SFRSYM    DATA     BYTE      S0RELL
      000000A0H.2 SFRSYM    DATA     BIT       P22
      00000090H.3 SFRSYM    DATA     BIT       P13
      00000080H.4 SFRSYM    DATA     BIT       P04
      000000C8H.1 SFRSYM    DATA     BIT       PWM0IF
      0000009DH   SFRSYM    DATA     BYTE      S1RELL
      000000A0H.3 SFRSYM    DATA     BIT       P23
      00000090H.4 SFRSYM    DATA     BIT       P14
      00000080H.5 SFRSYM    DATA     BIT       P05
      000000C3H   SFRSYM    DATA     BYTE      PWM0DL
      00000090H.5 SFRSYM    DATA     BIT       P15
      000000A6H   SFRSYM    DATA     BYTE      OSTATUS
      000000C5H   SFRSYM    DATA     BYTE      PWM1DL
      000000A0H.5 SFRSYM    DATA     BIT       P25
LX51 LINKER/LOCATER V4.66.97.0                                                        03/28/2025  17:08:22  PAGE 20


      000000D8H.4 SFRSYM    DATA     BIT       PORF
      000000D8H   SFRSYM    DATA     BYTE      RSTSTAT
      000000CFH   SFRSYM    DATA     BYTE      PWM2DL
      000000A0H.6 SFRSYM    DATA     BIT       P26
      000000C8H.7 SFRSYM    DATA     BIT       PWM0EN
      000000A0H.7 SFRSYM    DATA     BIT       P27
      000000A8H.5 SFRSYM    DATA     BIT       EPWM
      000000D8H.5 SFRSYM    DATA     BIT       LVRF
      000000F8H   SFRSYM    DATA     BYTE      CLKCON
      000000CCH   SFRSYM    DATA     BYTE      PWM0PH
      000000CEH   SFRSYM    DATA     BYTE      PWM1PH
      000000B8H.5 SFRSYM    DATA     BIT       I2CINTEN
      000000C2H   SFRSYM    DATA     BYTE      PWM2PH
      000000F0H   SFRSYM    DATA     BYTE      B
      000000EEH   SFRSYM    DATA     BYTE      RCHDIV
      000000CBH   SFRSYM    DATA     BYTE      PWM0PL
      000000CDH   SFRSYM    DATA     BYTE      PWM1PL
      000000C1H   SFRSYM    DATA     BYTE      PWM2PL
      000000F7H   SFRSYM    DATA     BYTE      ADCSPW
      000000F8H.1 SFRSYM    DATA     BIT       XCLKEN
      000000E0H   SFRSYM    DATA     BYTE      ACC
      000000DDH   SFRSYM    DATA     BYTE      LVDCON
      000000A8H.4 SFRSYM    DATA     BIT       ES0
      000000A9H   SFRSYM    DATA     BYTE      IP0
      000000A8H.1 SFRSYM    DATA     BIT       ET0
      000000A8H.2 SFRSYM    DATA     BIT       ES1
      000000F6H   SFRSYM    DATA     BYTE      ADCCSTAT
      000000B9H   SFRSYM    DATA     BYTE      IP1
      000000A8H.3 SFRSYM    DATA     BIT       ET1
      00000098H.0 SFRSYM    DATA     BIT       RI0
      000000C8H.0 SFRSYM    DATA     BIT       PWM0SS
      00000098H.1 SFRSYM    DATA     BIT       TI0
      000000A8H.0 SFRSYM    DATA     BIT       EX0
      000000D0H.0 SFRSYM    DATA     BIT       P
      000000B8H.3 SFRSYM    DATA     BIT       EFCINTEN
      000000A2H   SFRSYM    DATA     BYTE      OINTEN
      00000098H.7 SFRSYM    DATA     BIT       SM0
      00000098H.6 SFRSYM    DATA     BIT       SM1
      000000FEH   SFRSYM    DATA     BYTE      ADCCDR0
      000000FFH   SFRSYM    DATA     BYTE      ADCCDR1
      000000D0H.3 SFRSYM    DATA     BIT       RS0
      000000ACH   SFRSYM    DATA     BYTE      ADCGCR0
      000000D0H.4 SFRSYM    DATA     BIT       RS1
      000000ADH   SFRSYM    DATA     BYTE      ADCGCR1
      000000B4H   SFRSYM    DATA     BYTE      ADCGCR2
      000000B5H   SFRSYM    DATA     BYTE      ADCGCR3
      000000F8H.3 SFRSYM    DATA     BIT       RC32KEN
      000000DEH   SFRSYM    DATA     BYTE      PCLK0
      000000DFH   SFRSYM    DATA     BYTE      PCLK1
      00000083H   SFRSYM    DATA     BYTE      DPH
      000000E9H   SFRSYM    DATA     BYTE      P0IEN
      000000F5H   SFRSYM    DATA     BYTE      ADCHL
      000000F8H.2 SFRSYM    DATA     BIT       RC16MEN
      000000EAH   SFRSYM    DATA     BYTE      P1IEN
      000000EBH   SFRSYM    DATA     BYTE      P2IEN
      000000B6H   SFRSYM    DATA     WORD      ADCDR
      000000B3H   SFRSYM    DATA     BYTE      XTHCTR
      00000082H   SFRSYM    DATA     BYTE      DPL
      00000099H   SFRSYM    DATA     BYTE      S0BUF
      0000009CH   SFRSYM    DATA     BYTE      S1BUF
      000000F9H   SFRSYM    DATA     BYTE      P0OEN
      000000B8H.0 SFRSYM    DATA     BIT       GTIM0INTEN
      000000D9H   SFRSYM    DATA     BYTE      SYSDIV
      00000098H   SFRSYM    DATA     BYTE      S0CON
      000000FAH   SFRSYM    DATA     BYTE      P1OEN
LX51 LINKER/LOCATER V4.66.97.0                                                        03/28/2025  17:08:22  PAGE 21


      000000B8H.2 SFRSYM    DATA     BIT       GTIM1INTEN
      000000A3H   SFRSYM    DATA     BYTE      OINTUS
      000000BEH   SFRSYM    DATA     BYTE      RCHTRIMH
      000000F8H.0 SFRSYM    DATA     BIT       SYSSEL
      0000009BH   SFRSYM    DATA     BYTE      S1CON
      000000FBH   SFRSYM    DATA     BYTE      P2OEN
      000000B8H.6 SFRSYM    DATA     BIT       GTIM2INTEN
      000000BDH   SFRSYM    DATA     BYTE      LDOTRIMH
      00000092H   SFRSYM    DATA     BYTE      DPS
      0000009FH   SFRSYM    DATA     BYTE      RCLTRIMH
      000000BFH   SFRSYM    DATA     BYTE      RCHTRIML
      000000D3H   SFRSYM    DATA     BYTE      ODATA
      00000091H   SFRSYM    DATA     BYTE      LDOTRIML
      000000BCH   SFRSYM    DATA     BYTE      RCLTRIML
      000000E1H   SFRSYM    DATA     BYTE      P0IRQ
      000000B8H.1 SFRSYM    DATA     BIT       SPIINTEN
      000000E2H   SFRSYM    DATA     BYTE      P1IRQ
      000000E3H   SFRSYM    DATA     BYTE      P2IRQ
      000000D2H   SFRSYM    DATA     BYTE      OADRH
      000000B8H.7 SFRSYM    DATA     BIT       UART2INTEN
      000000F0H.0 SFRSYM    DATA     BIT       B0
      000000F0H.1 SFRSYM    DATA     BIT       B1
      000000F0H.2 SFRSYM    DATA     BIT       B2
      000000D1H   SFRSYM    DATA     BYTE      OADRL
      000000F0H.3 SFRSYM    DATA     BIT       B3
      000000F0H.4 SFRSYM    DATA     BIT       B4
      000000D0H.5 SFRSYM    DATA     BIT       F0
      000000F0H.5 SFRSYM    DATA     BIT       B5
      000000D0H.1 SFRSYM    DATA     BIT       F1
      000000AFH   SFRSYM    DATA     BYTE      REMAP
      000000F0H.6 SFRSYM    DATA     BIT       B6
      000000E0H.0 SFRSYM    DATA     BIT       ACC0
      000000A1H   SFRSYM    DATA     BYTE      OUS
      000000C8H.6 SFRSYM    DATA     BIT       PWM0S
      000000F0H.7 SFRSYM    DATA     BIT       B7
      000000E0H.1 SFRSYM    DATA     BIT       ACC1
      000000F8H.4 SFRSYM    DATA     BIT       XCLKF
      000000E0H.2 SFRSYM    DATA     BIT       ACC2
      0000008EH   SFRSYM    DATA     BYTE      PDSEL
      000000E0H.3 SFRSYM    DATA     BIT       ACC3
      000000D0H   SFRSYM    DATA     BYTE      PSW
      000000E0H.4 SFRSYM    DATA     BIT       ACC4
      00000098H.2 SFRSYM    DATA     BIT       RB80
      000000E0H.5 SFRSYM    DATA     BIT       ACC5
      000000FDH   SFRSYM    DATA     BYTE      ADCVREF
      000000E0H.6 SFRSYM    DATA     BIT       ACC6

      0100104DH   BLOCK     CODE     ---       LVL=0
      0200006DH   SYMBOL    XDATA    DWORD     system_clk_hz
      01001053H   BLOCK     CODE     NEAR LAB  LVL=1
      00000007H   SYMBOL    DATA     BYTE      system_clk_mhz
      ---         BLOCKEND  ---      ---       LVL=1
      0100104DH   LINE      CODE     ---       #14
      01001053H   LINE      CODE     ---       #15
      01001053H   LINE      CODE     ---       #18
      01001067H   LINE      CODE     ---       #19
      01001067H   LINE      CODE     ---       #21
      01001067H   LINE      CODE     ---       #23
      01001078H   LINE      CODE     ---       #25
      01001078H   LINE      CODE     ---       #27
      0100107AH   LINE      CODE     ---       #29
      0100107DH   LINE      CODE     ---       #30
      01001080H   LINE      CODE     ---       #32
      ---         BLOCKEND  ---      ---       LVL=0

LX51 LINKER/LOCATER V4.66.97.0                                                        03/28/2025  17:08:22  PAGE 22


      010010B2H   BLOCK     CODE     ---       LVL=0
      00000006H   SYMBOL    DATA     WORD      page_addr
      010010B2H   BLOCK     CODE     NEAR LAB  LVL=1
      00000020H.0 SYMBOL    BIT      BIT       temp
      ---         BLOCKEND  ---      ---       LVL=1
      010010B2H   LINE      CODE     ---       #34
      010010B2H   LINE      CODE     ---       #35
      010010B2H   LINE      CODE     ---       #37
      010010B6H   LINE      CODE     ---       #38
      010010B8H   LINE      CODE     ---       #40
      010010BBH   LINE      CODE     ---       #41
      010010BEH   LINE      CODE     ---       #43
      010010C2H   LINE      CODE     ---       #44
      010010C5H   LINE      CODE     ---       #45
      010010C8H   LINE      CODE     ---       #47
      010010CDH   LINE      CODE     ---       #49
      010010D0H   LINE      CODE     ---       #51
      010010D5H   LINE      CODE     ---       #53
      010010D8H   LINE      CODE     ---       #55
      010010DBH   LINE      CODE     ---       #57
      010010DFH   LINE      CODE     ---       #58
      ---         BLOCKEND  ---      ---       LVL=0
      00000006H   SYMBOL    DATA     WORD      addr
      00000005H   SYMBOL    DATA     BYTE      value

      01000E79H   BLOCK     CODE     ---       LVL=0
      02000078H   SYMBOL    XDATA    WORD      addr
      0200007AH   SYMBOL    XDATA    ---       buff
      0200007DH   SYMBOL    XDATA    DWORD     length
      01000E85H   BLOCK     CODE     NEAR LAB  LVL=1
      00000020H.0 SYMBOL    BIT      BIT       temp
      ---         BLOCKEND  ---      ---       LVL=1
      01000E79H   LINE      CODE     ---       #88
      01000E85H   LINE      CODE     ---       #89
      01000E85H   LINE      CODE     ---       #91
      01000E89H   LINE      CODE     ---       #92
      01000E8BH   LINE      CODE     ---       #94
      01000E8EH   LINE      CODE     ---       #95
      01000E91H   LINE      CODE     ---       #97
      01000E9FH   LINE      CODE     ---       #98
      01000E9FH   LINE      CODE     ---       #99
      01000EAFH   LINE      CODE     ---       #100
      01000EBEH   LINE      CODE     ---       #101
      01000EC1H   LINE      CODE     ---       #102
      01000EC4H   LINE      CODE     ---       #104
      01000EC9H   LINE      CODE     ---       #106
      01000ECCH   LINE      CODE     ---       #108
      01000ED1H   LINE      CODE     ---       #110
      01000ED4H   LINE      CODE     ---       #111
      01000ED6H   LINE      CODE     ---       #113
      01000ED9H   LINE      CODE     ---       #115
      01000EDDH   LINE      CODE     ---       #116
      ---         BLOCKEND  ---      ---       LVL=0

      01001140H   BLOCK     CODE     ---       LVL=0
      00000082H   SYMBOL    DATA     WORD      addr
      01001144H   BLOCK     CODE     NEAR LAB  LVL=1
      00000007H   SYMBOL    DATA     BYTE      value
      ---         BLOCKEND  ---      ---       LVL=1
      01001140H   LINE      CODE     ---       #118
      01001144H   LINE      CODE     ---       #119
      01001144H   LINE      CODE     ---       #122
      01001147H   LINE      CODE     ---       #124
      01001147H   LINE      CODE     ---       #126
      ---         BLOCKEND  ---      ---       LVL=0
LX51 LINKER/LOCATER V4.66.97.0                                                        03/28/2025  17:08:22  PAGE 23



      01000CB1H   BLOCK     CODE     ---       LVL=0
      02000078H   SYMBOL    XDATA    WORD      addr
      0200007AH   SYMBOL    XDATA    ---       buff
      0200007DH   SYMBOL    XDATA    DWORD     length
      01000CBDH   BLOCK     CODE     NEAR LAB  LVL=1
      02000081H   SYMBOL    XDATA    DWORD     index
      ---         BLOCKEND  ---      ---       LVL=1
      01000CB1H   LINE      CODE     ---       #128
      01000CBDH   LINE      CODE     ---       #129
      01000CBDH   LINE      CODE     ---       #132
      01000CD9H   LINE      CODE     ---       #133
      01000CD9H   LINE      CODE     ---       #134
      01000D08H   LINE      CODE     ---       #135
      01000D23H   LINE      CODE     ---       #137
      ---         BLOCKEND  ---      ---       LVL=0

      01001081H   BLOCK     CODE     ---       LVL=0
      02000089H   SYMBOL    XDATA    ---       buff
      01001087H   BLOCK     CODE     NEAR LAB  LVL=1
      00000007H   SYMBOL    DATA     BYTE      i
      ---         BLOCKEND  ---      ---       LVL=1
      01001081H   LINE      CODE     ---       #150
      01001087H   LINE      CODE     ---       #151
      01001087H   LINE      CODE     ---       #152
      01001089H   LINE      CODE     ---       #154
      01001093H   LINE      CODE     ---       #155
      01001093H   LINE      CODE     ---       #156
      010010AEH   LINE      CODE     ---       #157
      010010B1H   LINE      CODE     ---       #159
      ---         BLOCKEND  ---      ---       LVL=0

      01000A04H   BLOCK     CODE     ---       LVL=0
      00000001H   SYMBOL    DATA     ---       buff
      01000A04H   BLOCK     CODE     NEAR LAB  LVL=1
      02000089H   SYMBOL    XDATA    DWORD     temp
      ---         BLOCKEND  ---      ---       LVL=1
      01000A04H   LINE      CODE     ---       #162
      01000A04H   LINE      CODE     ---       #163
      01000A04H   LINE      CODE     ---       #164
      01000A0EH   LINE      CODE     ---       #165
      01000A1AH   LINE      CODE     ---       #167
      01000A29H   LINE      CODE     ---       #168
      01000A3BH   LINE      CODE     ---       #169
      01000A4DH   LINE      CODE     ---       #170
      01000A5AH   LINE      CODE     ---       #172
      01000A69H   LINE      CODE     ---       #173
      01000A76H   LINE      CODE     ---       #175
      01000A85H   LINE      CODE     ---       #176
      01000A92H   LINE      CODE     ---       #177
      01000AA1H   LINE      CODE     ---       #178
      01000AAEH   LINE      CODE     ---       #180
      01000ABDH   LINE      CODE     ---       #181
      ---         BLOCKEND  ---      ---       LVL=0

      01000EDEH   BLOCK     CODE     ---       LVL=0
      00000001H   SYMBOL    DATA     ---       buff
      01000EDEH   BLOCK     CODE     NEAR LAB  LVL=1
      02000089H   SYMBOL    XDATA    DWORD     temp
      ---         BLOCKEND  ---      ---       LVL=1
      01000EDEH   LINE      CODE     ---       #186
      01000EDEH   LINE      CODE     ---       #187
      01000EDEH   LINE      CODE     ---       #188
      01000EE8H   LINE      CODE     ---       #189
      01000EF4H   LINE      CODE     ---       #190
LX51 LINKER/LOCATER V4.66.97.0                                                        03/28/2025  17:08:22  PAGE 24


      01000F03H   LINE      CODE     ---       #191
      01000F15H   LINE      CODE     ---       #192
      01000F27H   LINE      CODE     ---       #193
      ---         BLOCKEND  ---      ---       LVL=0

      ---         MODULE    ---      ---       UART0
      020000C5H   PUBLIC    XDATA    ---       uart0_func
      020000C4H   PUBLIC    XDATA    BYTE      uart0_tx_flag
      0100001CH   PUBLIC    CODE     ---       _putchar
      01001148H   PUBLIC    CODE     ---       uart0_recv_byte
      01001102H   PUBLIC    CODE     ---       _uart0_send_byte
      01001118H   PUBLIC    CODE     ---       _uart0_irq_init
      01001016H   PUBLIC    CODE     ---       _uart0_init
      01000F85H   PUBLIC    CODE     ---       UART0_IRQHandler
      00000098H.3 SFRSYM    DATA     BIT       TB80
      000000E0H.7 SFRSYM    DATA     BIT       ACC7
      00000080H   SFRSYM    DATA     BYTE      P0
      00000090H   SFRSYM    DATA     BYTE      P1
      000000A0H   SFRSYM    DATA     BYTE      P2
      00000098H.5 SFRSYM    DATA     BIT       SM20
      000000B2H   SFRSYM    DATA     BYTE      ESTCR
      000000B1H   SFRSYM    DATA     BYTE      CLKST
      000000D0H.6 SFRSYM    DATA     BIT       AC
      000000D8H.3 SFRSYM    DATA     BIT       ERSTF
      000000E6H   SFRSYM    DATA     BYTE      PRESET0
      000000D4H   SFRSYM    DATA     BYTE      OCTRL
      000000A8H.7 SFRSYM    DATA     BIT       EA
      0000008FH   SFRSYM    DATA     BYTE      POREN
      000000C8H   SFRSYM    DATA     BYTE      PWM0CON
      000000E7H   SFRSYM    DATA     BYTE      PRESET1
      000000C9H   SFRSYM    DATA     BYTE      PWM1CON
      00000086H   SFRSYM    DATA     BYTE      BEEPCTR
      000000CAH   SFRSYM    DATA     BYTE      PWM2CON
      000000B8H.4 SFRSYM    DATA     BIT       LPTIMINTEN
      000000ABH   SFRSYM    DATA     BYTE      P0AH
      000000B0H   SFRSYM    DATA     BYTE      P1AH
      000000E8H   SFRSYM    DATA     BYTE      P2AH
      000000F8H.6 SFRSYM    DATA     BIT       RC32KF
      000000A8H   SFRSYM    DATA     BYTE      IEN0
      000000A7H   SFRSYM    DATA     BYTE      OPSET
      000000A4H   SFRSYM    DATA     BYTE      P0AL
      000000B8H   SFRSYM    DATA     BYTE      IEN1
      000000A8H.6 SFRSYM    DATA     BIT       EADC
      00000085H   SFRSYM    DATA     BYTE      DPH1
      000000AEH   SFRSYM    DATA     BYTE      P1AL
      0000009AH   SFRSYM    DATA     BYTE      IEN2
      000000C0H   SFRSYM    DATA     BYTE      P2AL
      000000B6H   SFRSYM    DATA     BYTE      ADCDR0
      000000F8H.5 SFRSYM    DATA     BIT       RC16MF
      000000B7H   SFRSYM    DATA     BYTE      ADCDR1
      00000084H   SFRSYM    DATA     BYTE      DPL1
      000000D6H   SFRSYM    DATA     BYTE      P0OD
      000000DBH   SFRSYM    DATA     BYTE      P1OD
      000000D5H   SFRSYM    DATA     BYTE      P0PD
      00000098H.4 SFRSYM    DATA     BIT       REN0
      000000ECH   SFRSYM    DATA     BYTE      P2OD
      000000DAH   SFRSYM    DATA     BYTE      P1PD
      000000E4H   SFRSYM    DATA     BYTE      P2PD
      000000D7H   SFRSYM    DATA     BYTE      P0CS
      00000097H   SFRSYM    DATA     BYTE      P0DR
      0000009EH   SFRSYM    DATA     BYTE      EUARTEN
      000000DCH   SFRSYM    DATA     BYTE      P1CS
      000000E5H   SFRSYM    DATA     BYTE      P1DR
      000000F4H   SFRSYM    DATA     BYTE      P2CS
      000000FCH   SFRSYM    DATA     BYTE      P2DR
LX51 LINKER/LOCATER V4.66.97.0                                                        03/28/2025  17:08:22  PAGE 25


      000000D0H.7 SFRSYM    DATA     BIT       CY
      000000D8H.0 SFRSYM    DATA     BIT       WDT0
      000000D8H.1 SFRSYM    DATA     BIT       WDT1
      000000D8H.2 SFRSYM    DATA     BIT       WDT2
      00000081H   SFRSYM    DATA     BYTE      SP
      000000F1H   SFRSYM    DATA     BYTE      P0PU
      000000F2H   SFRSYM    DATA     BYTE      P1PU
      000000D1H   SFRSYM    DATA     WORD      OADR
      000000F3H   SFRSYM    DATA     BYTE      P2PU
      00000093H   SFRSYM    DATA     BYTE      ADCIER
      000000A5H   SFRSYM    DATA     BYTE      OSEC
      000000D8H.6 SFRSYM    DATA     BIT       WDEN
      000000BAH   SFRSYM    DATA     BYTE      S0RELH
      00000080H.0 SFRSYM    DATA     BIT       P00
      000000D8H.7 SFRSYM    DATA     BIT       WDOF
      000000BBH   SFRSYM    DATA     BYTE      S1RELH
      00000090H.0 SFRSYM    DATA     BIT       P10
      00000080H.1 SFRSYM    DATA     BIT       P01
      00000087H   SFRSYM    DATA     BYTE      PCON
      000000C4H   SFRSYM    DATA     BYTE      PWM0DH
      000000A0H.0 SFRSYM    DATA     BIT       P20
      00000090H.1 SFRSYM    DATA     BIT       P11
      00000080H.2 SFRSYM    DATA     BIT       P02
      000000C6H   SFRSYM    DATA     BYTE      PWM1DH
      00000090H.2 SFRSYM    DATA     BIT       P12
      00000080H.3 SFRSYM    DATA     BIT       P03
      000000C7H   SFRSYM    DATA     BYTE      PWM2DH
      000000C8H.2 SFRSYM    DATA     BIT       PWM0IE
      000000AAH   SFRSYM    DATA     BYTE      S0RELL
      000000A0H.2 SFRSYM    DATA     BIT       P22
      00000090H.3 SFRSYM    DATA     BIT       P13
      00000080H.4 SFRSYM    DATA     BIT       P04
      000000C8H.1 SFRSYM    DATA     BIT       PWM0IF
      0000009DH   SFRSYM    DATA     BYTE      S1RELL
      000000A0H.3 SFRSYM    DATA     BIT       P23
      00000090H.4 SFRSYM    DATA     BIT       P14
      00000080H.5 SFRSYM    DATA     BIT       P05
      000000C3H   SFRSYM    DATA     BYTE      PWM0DL
      00000090H.5 SFRSYM    DATA     BIT       P15
      000000A6H   SFRSYM    DATA     BYTE      OSTATUS
      000000C5H   SFRSYM    DATA     BYTE      PWM1DL
      000000A0H.5 SFRSYM    DATA     BIT       P25
      000000D8H.4 SFRSYM    DATA     BIT       PORF
      000000D8H   SFRSYM    DATA     BYTE      RSTSTAT
      000000CFH   SFRSYM    DATA     BYTE      PWM2DL
      000000A0H.6 SFRSYM    DATA     BIT       P26
      000000C8H.7 SFRSYM    DATA     BIT       PWM0EN
      000000A0H.7 SFRSYM    DATA     BIT       P27
      000000A8H.5 SFRSYM    DATA     BIT       EPWM
      000000D8H.5 SFRSYM    DATA     BIT       LVRF
      000000F8H   SFRSYM    DATA     BYTE      CLKCON
      000000CCH   SFRSYM    DATA     BYTE      PWM0PH
      000000CEH   SFRSYM    DATA     BYTE      PWM1PH
      000000B8H.5 SFRSYM    DATA     BIT       I2CINTEN
      000000C2H   SFRSYM    DATA     BYTE      PWM2PH
      000000F0H   SFRSYM    DATA     BYTE      B
      000000EEH   SFRSYM    DATA     BYTE      RCHDIV
      000000CBH   SFRSYM    DATA     BYTE      PWM0PL
      000000CDH   SFRSYM    DATA     BYTE      PWM1PL
      000000C1H   SFRSYM    DATA     BYTE      PWM2PL
      000000F7H   SFRSYM    DATA     BYTE      ADCSPW
      000000F8H.1 SFRSYM    DATA     BIT       XCLKEN
      000000E0H   SFRSYM    DATA     BYTE      ACC
      000000DDH   SFRSYM    DATA     BYTE      LVDCON
      000000A8H.4 SFRSYM    DATA     BIT       ES0
LX51 LINKER/LOCATER V4.66.97.0                                                        03/28/2025  17:08:22  PAGE 26


      000000A9H   SFRSYM    DATA     BYTE      IP0
      000000A8H.1 SFRSYM    DATA     BIT       ET0
      000000A8H.2 SFRSYM    DATA     BIT       ES1
      000000F6H   SFRSYM    DATA     BYTE      ADCCSTAT
      000000B9H   SFRSYM    DATA     BYTE      IP1
      000000A8H.3 SFRSYM    DATA     BIT       ET1
      00000098H.0 SFRSYM    DATA     BIT       RI0
      000000C8H.0 SFRSYM    DATA     BIT       PWM0SS
      00000098H.1 SFRSYM    DATA     BIT       TI0
      000000A8H.0 SFRSYM    DATA     BIT       EX0
      000000D0H.0 SFRSYM    DATA     BIT       P
      000000B8H.3 SFRSYM    DATA     BIT       EFCINTEN
      000000A2H   SFRSYM    DATA     BYTE      OINTEN
      00000098H.7 SFRSYM    DATA     BIT       SM0
      00000098H.6 SFRSYM    DATA     BIT       SM1
      000000FEH   SFRSYM    DATA     BYTE      ADCCDR0
      000000FFH   SFRSYM    DATA     BYTE      ADCCDR1
      000000D0H.3 SFRSYM    DATA     BIT       RS0
      000000ACH   SFRSYM    DATA     BYTE      ADCGCR0
      000000D0H.4 SFRSYM    DATA     BIT       RS1
      000000ADH   SFRSYM    DATA     BYTE      ADCGCR1
      000000B4H   SFRSYM    DATA     BYTE      ADCGCR2
      000000B5H   SFRSYM    DATA     BYTE      ADCGCR3
      000000F8H.3 SFRSYM    DATA     BIT       RC32KEN
      000000DEH   SFRSYM    DATA     BYTE      PCLK0
      000000DFH   SFRSYM    DATA     BYTE      PCLK1
      00000083H   SFRSYM    DATA     BYTE      DPH
      000000E9H   SFRSYM    DATA     BYTE      P0IEN
      000000F5H   SFRSYM    DATA     BYTE      ADCHL
      000000F8H.2 SFRSYM    DATA     BIT       RC16MEN
      000000EAH   SFRSYM    DATA     BYTE      P1IEN
      000000EBH   SFRSYM    DATA     BYTE      P2IEN
      000000B6H   SFRSYM    DATA     WORD      ADCDR
      000000B3H   SFRSYM    DATA     BYTE      XTHCTR
      00000082H   SFRSYM    DATA     BYTE      DPL
      00000099H   SFRSYM    DATA     BYTE      S0BUF
      0000009CH   SFRSYM    DATA     BYTE      S1BUF
      000000F9H   SFRSYM    DATA     BYTE      P0OEN
      000000B8H.0 SFRSYM    DATA     BIT       GTIM0INTEN
      000000D9H   SFRSYM    DATA     BYTE      SYSDIV
      00000098H   SFRSYM    DATA     BYTE      S0CON
      000000FAH   SFRSYM    DATA     BYTE      P1OEN
      000000B8H.2 SFRSYM    DATA     BIT       GTIM1INTEN
      000000A3H   SFRSYM    DATA     BYTE      OINTUS
      000000BEH   SFRSYM    DATA     BYTE      RCHTRIMH
      000000F8H.0 SFRSYM    DATA     BIT       SYSSEL
      0000009BH   SFRSYM    DATA     BYTE      S1CON
      000000FBH   SFRSYM    DATA     BYTE      P2OEN
      000000B8H.6 SFRSYM    DATA     BIT       GTIM2INTEN
      000000BDH   SFRSYM    DATA     BYTE      LDOTRIMH
      00000092H   SFRSYM    DATA     BYTE      DPS
      0000009FH   SFRSYM    DATA     BYTE      RCLTRIMH
      000000BFH   SFRSYM    DATA     BYTE      RCHTRIML
      000000D3H   SFRSYM    DATA     BYTE      ODATA
      00000091H   SFRSYM    DATA     BYTE      LDOTRIML
      000000BCH   SFRSYM    DATA     BYTE      RCLTRIML
      000000E1H   SFRSYM    DATA     BYTE      P0IRQ
      000000B8H.1 SFRSYM    DATA     BIT       SPIINTEN
      000000E2H   SFRSYM    DATA     BYTE      P1IRQ
      000000E3H   SFRSYM    DATA     BYTE      P2IRQ
      000000D2H   SFRSYM    DATA     BYTE      OADRH
      000000B8H.7 SFRSYM    DATA     BIT       UART2INTEN
      000000F0H.0 SFRSYM    DATA     BIT       B0
      000000F0H.1 SFRSYM    DATA     BIT       B1
      000000F0H.2 SFRSYM    DATA     BIT       B2
LX51 LINKER/LOCATER V4.66.97.0                                                        03/28/2025  17:08:22  PAGE 27


      000000D1H   SFRSYM    DATA     BYTE      OADRL
      000000F0H.3 SFRSYM    DATA     BIT       B3
      000000F0H.4 SFRSYM    DATA     BIT       B4
      000000D0H.5 SFRSYM    DATA     BIT       F0
      000000F0H.5 SFRSYM    DATA     BIT       B5
      000000D0H.1 SFRSYM    DATA     BIT       F1
      000000AFH   SFRSYM    DATA     BYTE      REMAP
      000000F0H.6 SFRSYM    DATA     BIT       B6
      000000E0H.0 SFRSYM    DATA     BIT       ACC0
      000000A1H   SFRSYM    DATA     BYTE      OUS
      000000C8H.6 SFRSYM    DATA     BIT       PWM0S
      000000F0H.7 SFRSYM    DATA     BIT       B7
      000000E0H.1 SFRSYM    DATA     BIT       ACC1
      000000F8H.4 SFRSYM    DATA     BIT       XCLKF
      000000E0H.2 SFRSYM    DATA     BIT       ACC2
      0000008EH   SFRSYM    DATA     BYTE      PDSEL
      000000E0H.3 SFRSYM    DATA     BIT       ACC3
      000000D0H   SFRSYM    DATA     BYTE      PSW
      000000E0H.4 SFRSYM    DATA     BIT       ACC4
      00000098H.2 SFRSYM    DATA     BIT       RB80
      000000E0H.5 SFRSYM    DATA     BIT       ACC5
      000000FDH   SFRSYM    DATA     BYTE      ADCVREF
      000000E0H.6 SFRSYM    DATA     BIT       ACC6
      01000D29H   SYMBOL    CODE     ---       _uart0_set_baud_rate

      01000F85H   BLOCK     CODE     ---       LVL=0
      01000F85H   LINE      CODE     ---       #23
      01000FA2H   LINE      CODE     ---       #25
      01000FA5H   LINE      CODE     ---       #26
      01000FA5H   LINE      CODE     ---       #27
      01000FAFH   LINE      CODE     ---       #28
      01000FAFH   LINE      CODE     ---       #29
      01000FB2H   LINE      CODE     ---       #30
      01000FB2H   LINE      CODE     ---       #32
      01000FB4H   LINE      CODE     ---       #33
      01000FB4H   LINE      CODE     ---       #43
      ---         BLOCKEND  ---      ---       LVL=0

      01000D29H   BLOCK     CODE     ---       LVL=0
      02000071H   SYMBOL    XDATA    DWORD     clk_hz
      02000075H   SYMBOL    XDATA    DWORD     baud_rate
      01000D2FH   BLOCK     CODE     NEAR LAB  LVL=1
      02000079H   SYMBOL    XDATA    DWORD     temp
      00000003H   SYMBOL    DATA     BYTE      MSbyte
      00000007H   SYMBOL    DATA     BYTE      LSbyte
      ---         BLOCKEND  ---      ---       LVL=1
      01000D29H   LINE      CODE     ---       #53
      01000D2FH   LINE      CODE     ---       #54
      01000D2FH   LINE      CODE     ---       #58
      01000D44H   LINE      CODE     ---       #59
      01000D6BH   LINE      CODE     ---       #60
      01000D85H   LINE      CODE     ---       #62
      01000D92H   LINE      CODE     ---       #63
      01000D98H   LINE      CODE     ---       #65
      01000D9DH   LINE      CODE     ---       #66
      01000D9FH   LINE      CODE     ---       #67
      ---         BLOCKEND  ---      ---       LVL=0

      01001016H   BLOCK     CODE     ---       LVL=0
      0200006DH   SYMBOL    XDATA    DWORD     baud_rate
      01001016H   LINE      CODE     ---       #76
      0100101CH   LINE      CODE     ---       #77
      0100101CH   LINE      CODE     ---       #79
      0100101FH   LINE      CODE     ---       #80
      01001022H   LINE      CODE     ---       #81
LX51 LINKER/LOCATER V4.66.97.0                                                        03/28/2025  17:08:22  PAGE 28


      01001025H   LINE      CODE     ---       #83
      0100102AH   LINE      CODE     ---       #85
      0100102CH   LINE      CODE     ---       #86
      0100102EH   LINE      CODE     ---       #88
      01001030H   LINE      CODE     ---       #89
      01001032H   LINE      CODE     ---       #91
      01001047H   LINE      CODE     ---       #92
      01001049H   LINE      CODE     ---       #94
      0100104CH   LINE      CODE     ---       #95
      ---         BLOCKEND  ---      ---       LVL=0

      01001118H   BLOCK     CODE     ---       LVL=0
      00000007H   SYMBOL    DATA     BYTE      irqstate
      00000001H   SYMBOL    DATA     ---       pfunc_recv
      01001118H   LINE      CODE     ---       #105
      01001118H   LINE      CODE     ---       #106
      01001118H   LINE      CODE     ---       #107
      0100111DH   LINE      CODE     ---       #108
      0100111DH   LINE      CODE     ---       #109
      0100111FH   LINE      CODE     ---       #110
      01001121H   LINE      CODE     ---       #112
      01001127H   LINE      CODE     ---       #113
      01001127H   LINE      CODE     ---       #115
      01001127H   LINE      CODE     ---       #116
      01001129H   LINE      CODE     ---       #117
      01001129H   LINE      CODE     ---       #118
      ---         BLOCKEND  ---      ---       LVL=0

      01001102H   BLOCK     CODE     ---       LVL=0
      00000007H   SYMBOL    DATA     CHAR      c
      01001102H   BLOCK     CODE     NEAR LAB  LVL=1
      00000004H   SYMBOL    DATA     WORD      timeout
      ---         BLOCKEND  ---      ---       LVL=1
      01001102H   LINE      CODE     ---       #127
      01001102H   LINE      CODE     ---       #128
      01001102H   LINE      CODE     ---       #131
      01001106H   LINE      CODE     ---       #133
      01001108H   LINE      CODE     ---       #143
      0100110BH   LINE      CODE     ---       #144
      0100110BH   LINE      CODE     ---       #145
      01001115H   LINE      CODE     ---       #146
      01001115H   LINE      CODE     ---       #147
      01001115H   LINE      CODE     ---       #148
      01001115H   LINE      CODE     ---       #149
      01001115H   LINE      CODE     ---       #151
      01001117H   LINE      CODE     ---       #153
      ---         BLOCKEND  ---      ---       LVL=0

      01001148H   BLOCK     CODE     ---       LVL=0
      01001148H   LINE      CODE     ---       #178
      01001148H   LINE      CODE     ---       #179
      01001148H   LINE      CODE     ---       #180
      0100114AH   LINE      CODE     ---       #181
      ---         BLOCKEND  ---      ---       LVL=0

      0100001CH   BLOCK     CODE     ---       LVL=0
      00000003H   SYMBOL    DATA     CHAR      c
      0100001CH   LINE      CODE     ---       #189
      0100001EH   LINE      CODE     ---       #190
      0100001EH   LINE      CODE     ---       #191
      ---         BLOCKEND  ---      ---       LVL=0

      ---         MODULE    ---      ---       APP
      0200006BH   PUBLIC    XDATA    WORD      tx_count
      02000069H   PUBLIC    XDATA    WORD      rx_count
LX51 LINKER/LOCATER V4.66.97.0                                                        03/28/2025  17:08:22  PAGE 29


      02000068H   PUBLIC    XDATA    BYTE      rx_flag
      02000048H   PUBLIC    XDATA    ---       uart0_tx_buf
      02000028H   PUBLIC    XDATA    ---       uart0_rx_buf
      02000014H   PUBLIC    XDATA    ---       write_data
      02000000H   PUBLIC    XDATA    ---       read_data
      01000DA0H   PUBLIC    CODE     ---       eflash_test
      01000B78H   PUBLIC    CODE     ---       eflash_sn_test
      0200006DH   PUBLIC    XDATA    BYTE      ?_eflash_page_check_bytes?BYTE
      01000710H   PUBLIC    CODE     ---       _eflash_page_check_bytes
      01000ACAH   PUBLIC    CODE     ---       _eflash_page_check_byte
      01000003H   PUBLIC    CODE     ---       uart_init
      010010E0H   PUBLIC    CODE     ---       uart0_rec_pro
      00000098H.3 SFRSYM    DATA     BIT       TB80
      000000E0H.7 SFRSYM    DATA     BIT       ACC7
      00000080H   SFRSYM    DATA     BYTE      P0
      00000090H   SFRSYM    DATA     BYTE      P1
      000000A0H   SFRSYM    DATA     BYTE      P2
      00000098H.5 SFRSYM    DATA     BIT       SM20
      000000B2H   SFRSYM    DATA     BYTE      ESTCR
      000000B1H   SFRSYM    DATA     BYTE      CLKST
      000000D0H.6 SFRSYM    DATA     BIT       AC
      000000D8H.3 SFRSYM    DATA     BIT       ERSTF
      000000E6H   SFRSYM    DATA     BYTE      PRESET0
      000000D4H   SFRSYM    DATA     BYTE      OCTRL
      000000A8H.7 SFRSYM    DATA     BIT       EA
      0000008FH   SFRSYM    DATA     BYTE      POREN
      000000C8H   SFRSYM    DATA     BYTE      PWM0CON
      000000E7H   SFRSYM    DATA     BYTE      PRESET1
      000000C9H   SFRSYM    DATA     BYTE      PWM1CON
      00000086H   SFRSYM    DATA     BYTE      BEEPCTR
      000000CAH   SFRSYM    DATA     BYTE      PWM2CON
      000000B8H.4 SFRSYM    DATA     BIT       LPTIMINTEN
      000000ABH   SFRSYM    DATA     BYTE      P0AH
      000000B0H   SFRSYM    DATA     BYTE      P1AH
      000000E8H   SFRSYM    DATA     BYTE      P2AH
      000000F8H.6 SFRSYM    DATA     BIT       RC32KF
      000000A8H   SFRSYM    DATA     BYTE      IEN0
      000000A7H   SFRSYM    DATA     BYTE      OPSET
      000000A4H   SFRSYM    DATA     BYTE      P0AL
      000000B8H   SFRSYM    DATA     BYTE      IEN1
      000000A8H.6 SFRSYM    DATA     BIT       EADC
      00000085H   SFRSYM    DATA     BYTE      DPH1
      000000AEH   SFRSYM    DATA     BYTE      P1AL
      0000009AH   SFRSYM    DATA     BYTE      IEN2
      000000C0H   SFRSYM    DATA     BYTE      P2AL
      000000B6H   SFRSYM    DATA     BYTE      ADCDR0
      000000F8H.5 SFRSYM    DATA     BIT       RC16MF
      000000B7H   SFRSYM    DATA     BYTE      ADCDR1
      00000084H   SFRSYM    DATA     BYTE      DPL1
      000000D6H   SFRSYM    DATA     BYTE      P0OD
      000000DBH   SFRSYM    DATA     BYTE      P1OD
      000000D5H   SFRSYM    DATA     BYTE      P0PD
      00000098H.4 SFRSYM    DATA     BIT       REN0
      000000ECH   SFRSYM    DATA     BYTE      P2OD
      000000DAH   SFRSYM    DATA     BYTE      P1PD
      000000E4H   SFRSYM    DATA     BYTE      P2PD
      000000D7H   SFRSYM    DATA     BYTE      P0CS
      00000097H   SFRSYM    DATA     BYTE      P0DR
      0000009EH   SFRSYM    DATA     BYTE      EUARTEN
      000000DCH   SFRSYM    DATA     BYTE      P1CS
      000000E5H   SFRSYM    DATA     BYTE      P1DR
      000000F4H   SFRSYM    DATA     BYTE      P2CS
      000000FCH   SFRSYM    DATA     BYTE      P2DR
      000000D0H.7 SFRSYM    DATA     BIT       CY
      000000D8H.0 SFRSYM    DATA     BIT       WDT0
LX51 LINKER/LOCATER V4.66.97.0                                                        03/28/2025  17:08:22  PAGE 30


      000000D8H.1 SFRSYM    DATA     BIT       WDT1
      000000D8H.2 SFRSYM    DATA     BIT       WDT2
      00000081H   SFRSYM    DATA     BYTE      SP
      000000F1H   SFRSYM    DATA     BYTE      P0PU
      000000F2H   SFRSYM    DATA     BYTE      P1PU
      000000D1H   SFRSYM    DATA     WORD      OADR
      000000F3H   SFRSYM    DATA     BYTE      P2PU
      00000093H   SFRSYM    DATA     BYTE      ADCIER
      000000A5H   SFRSYM    DATA     BYTE      OSEC
      000000D8H.6 SFRSYM    DATA     BIT       WDEN
      000000BAH   SFRSYM    DATA     BYTE      S0RELH
      00000080H.0 SFRSYM    DATA     BIT       P00
      000000D8H.7 SFRSYM    DATA     BIT       WDOF
      000000BBH   SFRSYM    DATA     BYTE      S1RELH
      00000090H.0 SFRSYM    DATA     BIT       P10
      00000080H.1 SFRSYM    DATA     BIT       P01
      00000087H   SFRSYM    DATA     BYTE      PCON
      000000C4H   SFRSYM    DATA     BYTE      PWM0DH
      000000A0H.0 SFRSYM    DATA     BIT       P20
      00000090H.1 SFRSYM    DATA     BIT       P11
      00000080H.2 SFRSYM    DATA     BIT       P02
      000000C6H   SFRSYM    DATA     BYTE      PWM1DH
      00000090H.2 SFRSYM    DATA     BIT       P12
      00000080H.3 SFRSYM    DATA     BIT       P03
      000000C7H   SFRSYM    DATA     BYTE      PWM2DH
      000000C8H.2 SFRSYM    DATA     BIT       PWM0IE
      000000AAH   SFRSYM    DATA     BYTE      S0RELL
      000000A0H.2 SFRSYM    DATA     BIT       P22
      00000090H.3 SFRSYM    DATA     BIT       P13
      00000080H.4 SFRSYM    DATA     BIT       P04
      000000C8H.1 SFRSYM    DATA     BIT       PWM0IF
      0000009DH   SFRSYM    DATA     BYTE      S1RELL
      000000A0H.3 SFRSYM    DATA     BIT       P23
      00000090H.4 SFRSYM    DATA     BIT       P14
      00000080H.5 SFRSYM    DATA     BIT       P05
      000000C3H   SFRSYM    DATA     BYTE      PWM0DL
      00000090H.5 SFRSYM    DATA     BIT       P15
      000000A6H   SFRSYM    DATA     BYTE      OSTATUS
      000000C5H   SFRSYM    DATA     BYTE      PWM1DL
      000000A0H.5 SFRSYM    DATA     BIT       P25
      000000D8H.4 SFRSYM    DATA     BIT       PORF
      000000D8H   SFRSYM    DATA     BYTE      RSTSTAT
      000000CFH   SFRSYM    DATA     BYTE      PWM2DL
      000000A0H.6 SFRSYM    DATA     BIT       P26
      000000C8H.7 SFRSYM    DATA     BIT       PWM0EN
      000000A0H.7 SFRSYM    DATA     BIT       P27
      000000A8H.5 SFRSYM    DATA     BIT       EPWM
      000000D8H.5 SFRSYM    DATA     BIT       LVRF
      000000F8H   SFRSYM    DATA     BYTE      CLKCON
      000000CCH   SFRSYM    DATA     BYTE      PWM0PH
      000000CEH   SFRSYM    DATA     BYTE      PWM1PH
      000000B8H.5 SFRSYM    DATA     BIT       I2CINTEN
      000000C2H   SFRSYM    DATA     BYTE      PWM2PH
      000000F0H   SFRSYM    DATA     BYTE      B
      000000EEH   SFRSYM    DATA     BYTE      RCHDIV
      000000CBH   SFRSYM    DATA     BYTE      PWM0PL
      000000CDH   SFRSYM    DATA     BYTE      PWM1PL
      000000C1H   SFRSYM    DATA     BYTE      PWM2PL
      000000F7H   SFRSYM    DATA     BYTE      ADCSPW
      000000F8H.1 SFRSYM    DATA     BIT       XCLKEN
      000000E0H   SFRSYM    DATA     BYTE      ACC
      000000DDH   SFRSYM    DATA     BYTE      LVDCON
      000000A8H.4 SFRSYM    DATA     BIT       ES0
      000000A9H   SFRSYM    DATA     BYTE      IP0
      000000A8H.1 SFRSYM    DATA     BIT       ET0
LX51 LINKER/LOCATER V4.66.97.0                                                        03/28/2025  17:08:22  PAGE 31


      000000A8H.2 SFRSYM    DATA     BIT       ES1
      000000F6H   SFRSYM    DATA     BYTE      ADCCSTAT
      000000B9H   SFRSYM    DATA     BYTE      IP1
      000000A8H.3 SFRSYM    DATA     BIT       ET1
      00000098H.0 SFRSYM    DATA     BIT       RI0
      000000C8H.0 SFRSYM    DATA     BIT       PWM0SS
      00000098H.1 SFRSYM    DATA     BIT       TI0
      000000A8H.0 SFRSYM    DATA     BIT       EX0
      000000D0H.0 SFRSYM    DATA     BIT       P
      000000B8H.3 SFRSYM    DATA     BIT       EFCINTEN
      000000A2H   SFRSYM    DATA     BYTE      OINTEN
      00000098H.7 SFRSYM    DATA     BIT       SM0
      00000098H.6 SFRSYM    DATA     BIT       SM1
      000000FEH   SFRSYM    DATA     BYTE      ADCCDR0
      000000FFH   SFRSYM    DATA     BYTE      ADCCDR1
      000000D0H.3 SFRSYM    DATA     BIT       RS0
      000000ACH   SFRSYM    DATA     BYTE      ADCGCR0
      000000D0H.4 SFRSYM    DATA     BIT       RS1
      000000ADH   SFRSYM    DATA     BYTE      ADCGCR1
      000000B4H   SFRSYM    DATA     BYTE      ADCGCR2
      000000B5H   SFRSYM    DATA     BYTE      ADCGCR3
      000000F8H.3 SFRSYM    DATA     BIT       RC32KEN
      000000DEH   SFRSYM    DATA     BYTE      PCLK0
      000000DFH   SFRSYM    DATA     BYTE      PCLK1
      00000083H   SFRSYM    DATA     BYTE      DPH
      000000E9H   SFRSYM    DATA     BYTE      P0IEN
      000000F5H   SFRSYM    DATA     BYTE      ADCHL
      000000F8H.2 SFRSYM    DATA     BIT       RC16MEN
      000000EAH   SFRSYM    DATA     BYTE      P1IEN
      000000EBH   SFRSYM    DATA     BYTE      P2IEN
      000000B6H   SFRSYM    DATA     WORD      ADCDR
      000000B3H   SFRSYM    DATA     BYTE      XTHCTR
      00000082H   SFRSYM    DATA     BYTE      DPL
      00000099H   SFRSYM    DATA     BYTE      S0BUF
      0000009CH   SFRSYM    DATA     BYTE      S1BUF
      000000F9H   SFRSYM    DATA     BYTE      P0OEN
      000000B8H.0 SFRSYM    DATA     BIT       GTIM0INTEN
      000000D9H   SFRSYM    DATA     BYTE      SYSDIV
      00000098H   SFRSYM    DATA     BYTE      S0CON
      000000FAH   SFRSYM    DATA     BYTE      P1OEN
      000000B8H.2 SFRSYM    DATA     BIT       GTIM1INTEN
      000000A3H   SFRSYM    DATA     BYTE      OINTUS
      000000BEH   SFRSYM    DATA     BYTE      RCHTRIMH
      000000F8H.0 SFRSYM    DATA     BIT       SYSSEL
      0000009BH   SFRSYM    DATA     BYTE      S1CON
      000000FBH   SFRSYM    DATA     BYTE      P2OEN
      000000B8H.6 SFRSYM    DATA     BIT       GTIM2INTEN
      000000BDH   SFRSYM    DATA     BYTE      LDOTRIMH
      00000092H   SFRSYM    DATA     BYTE      DPS
      0000009FH   SFRSYM    DATA     BYTE      RCLTRIMH
      000000BFH   SFRSYM    DATA     BYTE      RCHTRIML
      000000D3H   SFRSYM    DATA     BYTE      ODATA
      00000091H   SFRSYM    DATA     BYTE      LDOTRIML
      000000BCH   SFRSYM    DATA     BYTE      RCLTRIML
      000000E1H   SFRSYM    DATA     BYTE      P0IRQ
      000000B8H.1 SFRSYM    DATA     BIT       SPIINTEN
      000000E2H   SFRSYM    DATA     BYTE      P1IRQ
      000000E3H   SFRSYM    DATA     BYTE      P2IRQ
      000000D2H   SFRSYM    DATA     BYTE      OADRH
      000000B8H.7 SFRSYM    DATA     BIT       UART2INTEN
      000000F0H.0 SFRSYM    DATA     BIT       B0
      000000F0H.1 SFRSYM    DATA     BIT       B1
      000000F0H.2 SFRSYM    DATA     BIT       B2
      000000D1H   SFRSYM    DATA     BYTE      OADRL
      000000F0H.3 SFRSYM    DATA     BIT       B3
LX51 LINKER/LOCATER V4.66.97.0                                                        03/28/2025  17:08:22  PAGE 32


      000000F0H.4 SFRSYM    DATA     BIT       B4
      000000D0H.5 SFRSYM    DATA     BIT       F0
      000000F0H.5 SFRSYM    DATA     BIT       B5
      000000D0H.1 SFRSYM    DATA     BIT       F1
      000000AFH   SFRSYM    DATA     BYTE      REMAP
      000000F0H.6 SFRSYM    DATA     BIT       B6
      000000E0H.0 SFRSYM    DATA     BIT       ACC0
      000000A1H   SFRSYM    DATA     BYTE      OUS
      000000C8H.6 SFRSYM    DATA     BIT       PWM0S
      000000F0H.7 SFRSYM    DATA     BIT       B7
      000000E0H.1 SFRSYM    DATA     BIT       ACC1
      000000F8H.4 SFRSYM    DATA     BIT       XCLKF
      000000E0H.2 SFRSYM    DATA     BIT       ACC2
      0000008EH   SFRSYM    DATA     BYTE      PDSEL
      000000E0H.3 SFRSYM    DATA     BIT       ACC3
      000000D0H   SFRSYM    DATA     BYTE      PSW
      000000E0H.4 SFRSYM    DATA     BIT       ACC4
      00000098H.2 SFRSYM    DATA     BIT       RB80
      000000E0H.5 SFRSYM    DATA     BIT       ACC5
      000000FDH   SFRSYM    DATA     BYTE      ADCVREF
      000000E0H.6 SFRSYM    DATA     BIT       ACC6

      010010E0H   BLOCK     CODE     ---       LVL=0
      010010E0H   LINE      CODE     ---       #34
      010010E0H   LINE      CODE     ---       #35
      010010E0H   LINE      CODE     ---       #36
      010010FBH   LINE      CODE     ---       #37
      01001101H   LINE      CODE     ---       #38
      ---         BLOCKEND  ---      ---       LVL=0

      01000003H   BLOCK     CODE     ---       LVL=0
      01000003H   LINE      CODE     ---       #47
      01000003H   LINE      CODE     ---       #48
      01000003H   LINE      CODE     ---       #49
      01000008H   LINE      CODE     ---       #50
      01000011H   LINE      CODE     ---       #51
      ---         BLOCKEND  ---      ---       LVL=0

      01000ACAH   BLOCK     CODE     ---       LVL=0
      0200006DH   SYMBOL    XDATA    WORD      base_addr
      00000005H   SYMBOL    DATA     BYTE      start_page
      0200006FH   SYMBOL    XDATA    BYTE      num_page
      01000AD5H   BLOCK     CODE     NEAR LAB  LVL=1
      02000070H   SYMBOL    XDATA    WORD      i
      02000072H   SYMBOL    XDATA    BYTE      page
      ---         BLOCKEND  ---      ---       LVL=1
      01000ACAH   LINE      CODE     ---       #78
      01000AD5H   LINE      CODE     ---       #79
      01000AD5H   LINE      CODE     ---       #85
      01000AEBH   LINE      CODE     ---       #86
      01000AEBH   LINE      CODE     ---       #87
      01000AFFH   LINE      CODE     ---       #88
      01000B14H   LINE      CODE     ---       #89
      01000B14H   LINE      CODE     ---       #90
      01000B31H   LINE      CODE     ---       #91
      01000B31H   LINE      CODE     ---       #92
      01000B60H   LINE      CODE     ---       #93
      01000B62H   LINE      CODE     ---       #94
      01000B62H   LINE      CODE     ---       #95
      01000B6EH   LINE      CODE     ---       #97
      01000B77H   LINE      CODE     ---       #100
      ---         BLOCKEND  ---      ---       LVL=0

      01000710H   BLOCK     CODE     ---       LVL=0
      0200006DH   SYMBOL    XDATA    WORD      base_addr
LX51 LINKER/LOCATER V4.66.97.0                                                        03/28/2025  17:08:22  PAGE 33


      0200006FH   SYMBOL    XDATA    BYTE      w_val
      02000070H   SYMBOL    XDATA    DWORD     length
      0100071DH   BLOCK     CODE     NEAR LAB  LVL=1
      02000074H   SYMBOL    XDATA    DWORD     i
      ---         BLOCKEND  ---      ---       LVL=1
      01000710H   LINE      CODE     ---       #102
      0100071DH   LINE      CODE     ---       #103
      0100071DH   LINE      CODE     ---       #107
      01000720H   LINE      CODE     ---       #109
      0100073CH   LINE      CODE     ---       #110
      0100073CH   LINE      CODE     ---       #111
      01000755H   LINE      CODE     ---       #112
      01000755H   LINE      CODE     ---       #113
      01000778H   LINE      CODE     ---       #114
      0100077AH   LINE      CODE     ---       #115
      0100077AH   LINE      CODE     ---       #116
      01000795H   LINE      CODE     ---       #118
      010007B1H   LINE      CODE     ---       #119
      010007B1H   LINE      CODE     ---       #120
      010007C8H   LINE      CODE     ---       #121
      010007E3H   LINE      CODE     ---       #123
      01000800H   LINE      CODE     ---       #125
      0100082CH   LINE      CODE     ---       #126
      0100082CH   LINE      CODE     ---       #127
      01000848H   LINE      CODE     ---       #128
      01000848H   LINE      CODE     ---       #129
      01000863H   LINE      CODE     ---       #130
      01000863H   LINE      CODE     ---       #131
      01000886H   LINE      CODE     ---       #132
      01000886H   LINE      CODE     ---       #133
      01000886H   LINE      CODE     ---       #134
      010008A4H   LINE      CODE     ---       #135
      010008C0H   LINE      CODE     ---       #136
      010008C0H   LINE      CODE     ---       #137
      ---         BLOCKEND  ---      ---       LVL=0

      01000B78H   BLOCK     CODE     ---       LVL=0
      01000B78H   BLOCK     CODE     NEAR LAB  LVL=1
      0200006DH   SYMBOL    XDATA    ---       chip_sn
      0200007DH   SYMBOL    XDATA    ---       chip_UID
      02000085H   SYMBOL    XDATA    ---       chip_Vcap
      ---         BLOCKEND  ---      ---       LVL=1
      01000B78H   LINE      CODE     ---       #141
      01000B78H   LINE      CODE     ---       #142
      01000B78H   LINE      CODE     ---       #147
      01000B81H   LINE      CODE     ---       #148
      01000B8AH   LINE      CODE     ---       #149
      01000B93H   LINE      CODE     ---       #150
      01000BA4H   LINE      CODE     ---       #151
      01000BADH   LINE      CODE     ---       #154
      01000BB6H   LINE      CODE     ---       #155
      01000BBFH   LINE      CODE     ---       #156
      01000BC8H   LINE      CODE     ---       #157
      01000BD9H   LINE      CODE     ---       #158
      01000BE2H   LINE      CODE     ---       #160
      01000BEBH   LINE      CODE     ---       #161
      01000BF4H   LINE      CODE     ---       #162
      01000BFDH   LINE      CODE     ---       #163
      01000C0EH   LINE      CODE     ---       #164
      ---         BLOCKEND  ---      ---       LVL=0

      01000DA0H   BLOCK     CODE     ---       LVL=0
      01000DA0H   LINE      CODE     ---       #169
      01000DA0H   LINE      CODE     ---       #170
      01000DA0H   LINE      CODE     ---       #173
LX51 LINKER/LOCATER V4.66.97.0                                                        03/28/2025  17:08:22  PAGE 34


      01000DB5H   LINE      CODE     ---       #174
      01000DBEH   LINE      CODE     ---       #178
      01000DC7H   LINE      CODE     ---       #179
      01000DD1H   LINE      CODE     ---       #180
      01000DDAH   LINE      CODE     ---       #182
      01000DE5H   LINE      CODE     ---       #184
      01000DEEH   LINE      CODE     ---       #185
      01000E01H   LINE      CODE     ---       #187
      01000E0AH   LINE      CODE     ---       #191
      ---         BLOCKEND  ---      ---       LVL=0

      ---         MODULE    ---      ---       MAIN
      01001135H   PUBLIC    CODE     ---       main
      00000098H.3 SFRSYM    DATA     BIT       TB80
      000000E0H.7 SFRSYM    DATA     BIT       ACC7
      00000080H   SFRSYM    DATA     BYTE      P0
      00000090H   SFRSYM    DATA     BYTE      P1
      000000A0H   SFRSYM    DATA     BYTE      P2
      00000098H.5 SFRSYM    DATA     BIT       SM20
      000000B2H   SFRSYM    DATA     BYTE      ESTCR
      000000B1H   SFRSYM    DATA     BYTE      CLKST
      000000D0H.6 SFRSYM    DATA     BIT       AC
      000000D8H.3 SFRSYM    DATA     BIT       ERSTF
      000000E6H   SFRSYM    DATA     BYTE      PRESET0
      000000D4H   SFRSYM    DATA     BYTE      OCTRL
      000000A8H.7 SFRSYM    DATA     BIT       EA
      0000008FH   SFRSYM    DATA     BYTE      POREN
      000000C8H   SFRSYM    DATA     BYTE      PWM0CON
      000000E7H   SFRSYM    DATA     BYTE      PRESET1
      000000C9H   SFRSYM    DATA     BYTE      PWM1CON
      00000086H   SFRSYM    DATA     BYTE      BEEPCTR
      000000CAH   SFRSYM    DATA     BYTE      PWM2CON
      000000B8H.4 SFRSYM    DATA     BIT       LPTIMINTEN
      000000ABH   SFRSYM    DATA     BYTE      P0AH
      000000B0H   SFRSYM    DATA     BYTE      P1AH
      000000E8H   SFRSYM    DATA     BYTE      P2AH
      000000F8H.6 SFRSYM    DATA     BIT       RC32KF
      000000A8H   SFRSYM    DATA     BYTE      IEN0
      000000A7H   SFRSYM    DATA     BYTE      OPSET
      000000A4H   SFRSYM    DATA     BYTE      P0AL
      000000B8H   SFRSYM    DATA     BYTE      IEN1
      000000A8H.6 SFRSYM    DATA     BIT       EADC
      00000085H   SFRSYM    DATA     BYTE      DPH1
      000000AEH   SFRSYM    DATA     BYTE      P1AL
      0000009AH   SFRSYM    DATA     BYTE      IEN2
      000000C0H   SFRSYM    DATA     BYTE      P2AL
      000000B6H   SFRSYM    DATA     BYTE      ADCDR0
      000000F8H.5 SFRSYM    DATA     BIT       RC16MF
      000000B7H   SFRSYM    DATA     BYTE      ADCDR1
      00000084H   SFRSYM    DATA     BYTE      DPL1
      000000D6H   SFRSYM    DATA     BYTE      P0OD
      000000DBH   SFRSYM    DATA     BYTE      P1OD
      000000D5H   SFRSYM    DATA     BYTE      P0PD
      00000098H.4 SFRSYM    DATA     BIT       REN0
      000000ECH   SFRSYM    DATA     BYTE      P2OD
      000000DAH   SFRSYM    DATA     BYTE      P1PD
      000000E4H   SFRSYM    DATA     BYTE      P2PD
      000000D7H   SFRSYM    DATA     BYTE      P0CS
      00000097H   SFRSYM    DATA     BYTE      P0DR
      0000009EH   SFRSYM    DATA     BYTE      EUARTEN
      000000DCH   SFRSYM    DATA     BYTE      P1CS
      000000E5H   SFRSYM    DATA     BYTE      P1DR
      000000F4H   SFRSYM    DATA     BYTE      P2CS
      000000FCH   SFRSYM    DATA     BYTE      P2DR
      000000D0H.7 SFRSYM    DATA     BIT       CY
LX51 LINKER/LOCATER V4.66.97.0                                                        03/28/2025  17:08:22  PAGE 35


      000000D8H.0 SFRSYM    DATA     BIT       WDT0
      000000D8H.1 SFRSYM    DATA     BIT       WDT1
      000000D8H.2 SFRSYM    DATA     BIT       WDT2
      00000081H   SFRSYM    DATA     BYTE      SP
      000000F1H   SFRSYM    DATA     BYTE      P0PU
      000000F2H   SFRSYM    DATA     BYTE      P1PU
      000000D1H   SFRSYM    DATA     WORD      OADR
      000000F3H   SFRSYM    DATA     BYTE      P2PU
      00000093H   SFRSYM    DATA     BYTE      ADCIER
      000000A5H   SFRSYM    DATA     BYTE      OSEC
      000000D8H.6 SFRSYM    DATA     BIT       WDEN
      000000BAH   SFRSYM    DATA     BYTE      S0RELH
      00000080H.0 SFRSYM    DATA     BIT       P00
      000000D8H.7 SFRSYM    DATA     BIT       WDOF
      000000BBH   SFRSYM    DATA     BYTE      S1RELH
      00000090H.0 SFRSYM    DATA     BIT       P10
      00000080H.1 SFRSYM    DATA     BIT       P01
      00000087H   SFRSYM    DATA     BYTE      PCON
      000000C4H   SFRSYM    DATA     BYTE      PWM0DH
      000000A0H.0 SFRSYM    DATA     BIT       P20
      00000090H.1 SFRSYM    DATA     BIT       P11
      00000080H.2 SFRSYM    DATA     BIT       P02
      000000C6H   SFRSYM    DATA     BYTE      PWM1DH
      00000090H.2 SFRSYM    DATA     BIT       P12
      00000080H.3 SFRSYM    DATA     BIT       P03
      000000C7H   SFRSYM    DATA     BYTE      PWM2DH
      000000C8H.2 SFRSYM    DATA     BIT       PWM0IE
      000000AAH   SFRSYM    DATA     BYTE      S0RELL
      000000A0H.2 SFRSYM    DATA     BIT       P22
      00000090H.3 SFRSYM    DATA     BIT       P13
      00000080H.4 SFRSYM    DATA     BIT       P04
      000000C8H.1 SFRSYM    DATA     BIT       PWM0IF
      0000009DH   SFRSYM    DATA     BYTE      S1RELL
      000000A0H.3 SFRSYM    DATA     BIT       P23
      00000090H.4 SFRSYM    DATA     BIT       P14
      00000080H.5 SFRSYM    DATA     BIT       P05
      000000C3H   SFRSYM    DATA     BYTE      PWM0DL
      00000090H.5 SFRSYM    DATA     BIT       P15
      000000A6H   SFRSYM    DATA     BYTE      OSTATUS
      000000C5H   SFRSYM    DATA     BYTE      PWM1DL
      000000A0H.5 SFRSYM    DATA     BIT       P25
      000000D8H.4 SFRSYM    DATA     BIT       PORF
      000000D8H   SFRSYM    DATA     BYTE      RSTSTAT
      000000CFH   SFRSYM    DATA     BYTE      PWM2DL
      000000A0H.6 SFRSYM    DATA     BIT       P26
      000000C8H.7 SFRSYM    DATA     BIT       PWM0EN
      000000A0H.7 SFRSYM    DATA     BIT       P27
      000000A8H.5 SFRSYM    DATA     BIT       EPWM
      000000D8H.5 SFRSYM    DATA     BIT       LVRF
      000000F8H   SFRSYM    DATA     BYTE      CLKCON
      000000CCH   SFRSYM    DATA     BYTE      PWM0PH
      000000CEH   SFRSYM    DATA     BYTE      PWM1PH
      000000B8H.5 SFRSYM    DATA     BIT       I2CINTEN
      000000C2H   SFRSYM    DATA     BYTE      PWM2PH
      000000F0H   SFRSYM    DATA     BYTE      B
      000000EEH   SFRSYM    DATA     BYTE      RCHDIV
      000000CBH   SFRSYM    DATA     BYTE      PWM0PL
      000000CDH   SFRSYM    DATA     BYTE      PWM1PL
      000000C1H   SFRSYM    DATA     BYTE      PWM2PL
      000000F7H   SFRSYM    DATA     BYTE      ADCSPW
      000000F8H.1 SFRSYM    DATA     BIT       XCLKEN
      000000E0H   SFRSYM    DATA     BYTE      ACC
      000000DDH   SFRSYM    DATA     BYTE      LVDCON
      000000A8H.4 SFRSYM    DATA     BIT       ES0
      000000A9H   SFRSYM    DATA     BYTE      IP0
LX51 LINKER/LOCATER V4.66.97.0                                                        03/28/2025  17:08:22  PAGE 36


      000000A8H.1 SFRSYM    DATA     BIT       ET0
      000000A8H.2 SFRSYM    DATA     BIT       ES1
      000000F6H   SFRSYM    DATA     BYTE      ADCCSTAT
      000000B9H   SFRSYM    DATA     BYTE      IP1
      000000A8H.3 SFRSYM    DATA     BIT       ET1
      00000098H.0 SFRSYM    DATA     BIT       RI0
      000000C8H.0 SFRSYM    DATA     BIT       PWM0SS
      00000098H.1 SFRSYM    DATA     BIT       TI0
      000000A8H.0 SFRSYM    DATA     BIT       EX0
      000000D0H.0 SFRSYM    DATA     BIT       P
      000000B8H.3 SFRSYM    DATA     BIT       EFCINTEN
      000000A2H   SFRSYM    DATA     BYTE      OINTEN
      00000098H.7 SFRSYM    DATA     BIT       SM0
      00000098H.6 SFRSYM    DATA     BIT       SM1
      000000FEH   SFRSYM    DATA     BYTE      ADCCDR0
      000000FFH   SFRSYM    DATA     BYTE      ADCCDR1
      000000D0H.3 SFRSYM    DATA     BIT       RS0
      000000ACH   SFRSYM    DATA     BYTE      ADCGCR0
      000000D0H.4 SFRSYM    DATA     BIT       RS1
      000000ADH   SFRSYM    DATA     BYTE      ADCGCR1
      000000B4H   SFRSYM    DATA     BYTE      ADCGCR2
      000000B5H   SFRSYM    DATA     BYTE      ADCGCR3
      000000F8H.3 SFRSYM    DATA     BIT       RC32KEN
      000000DEH   SFRSYM    DATA     BYTE      PCLK0
      000000DFH   SFRSYM    DATA     BYTE      PCLK1
      00000083H   SFRSYM    DATA     BYTE      DPH
      000000E9H   SFRSYM    DATA     BYTE      P0IEN
      000000F5H   SFRSYM    DATA     BYTE      ADCHL
      000000F8H.2 SFRSYM    DATA     BIT       RC16MEN
      000000EAH   SFRSYM    DATA     BYTE      P1IEN
      000000EBH   SFRSYM    DATA     BYTE      P2IEN
      000000B6H   SFRSYM    DATA     WORD      ADCDR
      000000B3H   SFRSYM    DATA     BYTE      XTHCTR
      00000082H   SFRSYM    DATA     BYTE      DPL
      00000099H   SFRSYM    DATA     BYTE      S0BUF
      0000009CH   SFRSYM    DATA     BYTE      S1BUF
      000000F9H   SFRSYM    DATA     BYTE      P0OEN
      000000B8H.0 SFRSYM    DATA     BIT       GTIM0INTEN
      000000D9H   SFRSYM    DATA     BYTE      SYSDIV
      00000098H   SFRSYM    DATA     BYTE      S0CON
      000000FAH   SFRSYM    DATA     BYTE      P1OEN
      000000B8H.2 SFRSYM    DATA     BIT       GTIM1INTEN
      000000A3H   SFRSYM    DATA     BYTE      OINTUS
      000000BEH   SFRSYM    DATA     BYTE      RCHTRIMH
      000000F8H.0 SFRSYM    DATA     BIT       SYSSEL
      0000009BH   SFRSYM    DATA     BYTE      S1CON
      000000FBH   SFRSYM    DATA     BYTE      P2OEN
      000000B8H.6 SFRSYM    DATA     BIT       GTIM2INTEN
      000000BDH   SFRSYM    DATA     BYTE      LDOTRIMH
      00000092H   SFRSYM    DATA     BYTE      DPS
      0000009FH   SFRSYM    DATA     BYTE      RCLTRIMH
      000000BFH   SFRSYM    DATA     BYTE      RCHTRIML
      000000D3H   SFRSYM    DATA     BYTE      ODATA
      00000091H   SFRSYM    DATA     BYTE      LDOTRIML
      000000BCH   SFRSYM    DATA     BYTE      RCLTRIML
      000000E1H   SFRSYM    DATA     BYTE      P0IRQ
      000000B8H.1 SFRSYM    DATA     BIT       SPIINTEN
      000000E2H   SFRSYM    DATA     BYTE      P1IRQ
      000000E3H   SFRSYM    DATA     BYTE      P2IRQ
      000000D2H   SFRSYM    DATA     BYTE      OADRH
      000000B8H.7 SFRSYM    DATA     BIT       UART2INTEN
      000000F0H.0 SFRSYM    DATA     BIT       B0
      000000F0H.1 SFRSYM    DATA     BIT       B1
      000000F0H.2 SFRSYM    DATA     BIT       B2
      000000D1H   SFRSYM    DATA     BYTE      OADRL
LX51 LINKER/LOCATER V4.66.97.0                                                        03/28/2025  17:08:22  PAGE 37


      000000F0H.3 SFRSYM    DATA     BIT       B3
      000000F0H.4 SFRSYM    DATA     BIT       B4
      000000D0H.5 SFRSYM    DATA     BIT       F0
      000000F0H.5 SFRSYM    DATA     BIT       B5
      000000D0H.1 SFRSYM    DATA     BIT       F1
      000000AFH   SFRSYM    DATA     BYTE      REMAP
      000000F0H.6 SFRSYM    DATA     BIT       B6
      000000E0H.0 SFRSYM    DATA     BIT       ACC0
      000000A1H   SFRSYM    DATA     BYTE      OUS
      000000C8H.6 SFRSYM    DATA     BIT       PWM0S
      000000F0H.7 SFRSYM    DATA     BIT       B7
      000000E0H.1 SFRSYM    DATA     BIT       ACC1
      000000F8H.4 SFRSYM    DATA     BIT       XCLKF
      000000E0H.2 SFRSYM    DATA     BIT       ACC2
      0000008EH   SFRSYM    DATA     BYTE      PDSEL
      000000E0H.3 SFRSYM    DATA     BIT       ACC3
      000000D0H   SFRSYM    DATA     BYTE      PSW
      000000E0H.4 SFRSYM    DATA     BIT       ACC4
      00000098H.2 SFRSYM    DATA     BIT       RB80
      000000E0H.5 SFRSYM    DATA     BIT       ACC5
      000000FDH   SFRSYM    DATA     BYTE      ADCVREF
      000000E0H.6 SFRSYM    DATA     BIT       ACC6

      01001135H   BLOCK     CODE     ---       LVL=0
      01001135H   LINE      CODE     ---       #14
      01001135H   LINE      CODE     ---       #15
      01001135H   LINE      CODE     ---       #16
      01001138H   LINE      CODE     ---       #18
      0100113BH   LINE      CODE     ---       #20
      0100113EH   LINE      CODE     ---       #22
      0100113EH   LINE      CODE     ---       #23
      0100113EH   LINE      CODE     ---       #25
      ---         BLOCKEND  ---      ---       LVL=0

      ---         MODULE    ---      ---       ?C_INIT
      01000C6CH   PUBLIC    CODE     ---       ?C_START

      ---         MODULE    ---      ---       ?C?CLDPTR
      01000026H   PUBLIC    CODE     ---       ?C?CLDPTR

      ---         MODULE    ---      ---       ?C?CLDOPTR
      0100003FH   PUBLIC    CODE     ---       ?C?CLDOPTR

      ---         MODULE    ---      ---       ?C?CSTPTR
      0100006CH   PUBLIC    CODE     ---       ?C?CSTPTR

      ---         MODULE    ---      ---       ?C?CSTOPTR
      0100007EH   PUBLIC    CODE     ---       ?C?CSTOPTR

      ---         MODULE    ---      ---       ?C?IILDX
      010000A0H   PUBLIC    CODE     ---       ?C?IILDX

      ---         MODULE    ---      ---       ?C?ILDIX
      010000B6H   PUBLIC    CODE     ---       ?C?ILDIX

      ---         MODULE    ---      ---       ?C?LADD
      010000CCH   PUBLIC    CODE     ---       ?C?LADD

      ---         MODULE    ---      ---       ?C?LMUL
      010000D9H   PUBLIC    CODE     ---       ?C?LMUL

      ---         MODULE    ---      ---       ?C?ULDIV
      01000164H   PUBLIC    CODE     ---       ?C?ULDIV

      ---         MODULE    ---      ---       ?C?LOR
LX51 LINKER/LOCATER V4.66.97.0                                                        03/28/2025  17:08:22  PAGE 38


      010001F6H   PUBLIC    CODE     ---       ?C?LOR

      ---         MODULE    ---      ---       ?C?ULCMP
      01000203H   PUBLIC    CODE     ---       ?C?ULCMP

      ---         MODULE    ---      ---       ?C?ULSHR
      01000214H   PUBLIC    CODE     ---       ?C?ULSHR

      ---         MODULE    ---      ---       ?C?LSHL
      01000227H   PUBLIC    CODE     ---       ?C?LSHL

      ---         MODULE    ---      ---       ?C?LLDOPTR
      0100023AH   PUBLIC    CODE     ---       ?C?LLDOPTR

      ---         MODULE    ---      ---       ?C?LLDXDATA
      0100026AH   PUBLIC    CODE     ---       ?C?LLDXDATA

      ---         MODULE    ---      ---       ?C?LLDXDATA0
      01000276H   PUBLIC    CODE     ---       ?C?LLDXDATA0

      ---         MODULE    ---      ---       ?C?LLDIXDATA
      0100028BH   PUBLIC    CODE     ---       ?C?LLDIXDATA
      01000282H   PUBLIC    CODE     ---       ?C?LLDIXDATA1
      01000284H   PUBLIC    CODE     ---       ?C?LLDIXDATA8

      ---         MODULE    ---      ---       ?C?LSTXDATA
      010002B7H   PUBLIC    CODE     ---       ?C?LSTXDATA

      ---         MODULE    ---      ---       ?C?LSTKXDATA
      010002C3H   PUBLIC    CODE     ---       ?C?LSTKXDATA

      ---         MODULE    ---      ---       ?C?PLDXDATA
      010002F4H   PUBLIC    CODE     ---       ?C?PLDXDATA

      ---         MODULE    ---      ---       ?C?PLDIXDATA
      010002FDH   PUBLIC    CODE     ---       ?C?PLDIXDATA

      ---         MODULE    ---      ---       ?C?PSTXDATA
      01000314H   PUBLIC    CODE     ---       ?C?PSTXDATA

      ---         MODULE    ---      ---       ?C?LCASE
      0100031DH   PUBLIC    CODE     ---       ?C?LCASE

      ---         MODULE    ---      ---       ?C?ICALL
      01000357H   PUBLIC    CODE     ---       ?C?ICALL
      0100035BH   PUBLIC    CODE     ---       ?C?ICALL2

      ---         MODULE    ---      ---       PRINTF
      02000094H   PUBLIC    XDATA    ---       ?_PRINTF517?BYTE
      02000094H   PUBLIC    XDATA    ---       ?_PRINTF?BYTE
      02000094H   PUBLIC    XDATA    ---       ?_SPRINTF517?BYTE
      02000094H   PUBLIC    XDATA    ---       ?_SPRINTF?BYTE
      01000416H   PUBLIC    CODE     ---       _PRINTF
      01000416H   PUBLIC    CODE     ---       _PRINTF517
      01000410H   PUBLIC    CODE     ---       _SPRINTF
      01000410H   PUBLIC    CODE     ---       _SPRINTF517

      ---         MODULE    ---      ---       ?C?LLDIDATA
      0100035DH   PUBLIC    CODE     ---       ?C?LLDIDATA

      ---         MODULE    ---      ---       ?C?LLDPDATA
      01000369H   PUBLIC    CODE     ---       ?C?LLDPDATA

      ---         MODULE    ---      ---       ?C?LLDCODE
      01000375H   PUBLIC    CODE     ---       ?C?LLDCODE
LX51 LINKER/LOCATER V4.66.97.0                                                        03/28/2025  17:08:22  PAGE 39



      ---         MODULE    ---      ---       ?C?CCASE
      01000385H   PUBLIC    CODE     ---       ?C?CCASE

Program Size: data=15.1 xdata=200 const=563 code=4425
LX51 RUN COMPLETE.  0 WARNING(S),  0 ERROR(S)
